:020000040800F2
:1000000000060020F5050008B51A0008311A00089E
:10001000891A0008311A00085D1A0008F70500085F
:10002000F7050008F7050008F7050008155B00084C
:10003000F7050008F7050008F7050008F7050008B0
:10004000F7050008F7050008F7050008F7050008A0
:10005000F7050008F70500080D5F0008395F000884
:10006000655F0008915F0008BD5F0008F7050008A4
:10007000F7050008F7050008F7050008F705000870
:10008000F7050008F7050008F7050008F705000860
:10009000F7050008F7050008F7050008E95F000804
:1000A000F7050008F7050008F7050008F705000840
:1000B000F7050008F7050008F7050008F705000830
:1000C000F7050008F7050008F7050008F705000820
:1000D000F7050008D5600008F7050008F7050008D7
:1000E0004D600008F7050008F7050008F70500084F
:1000F000F7050008F7050008F7050008F7050008F0
:10010000F7050008F7050008E9600008F705000892
:10011000F7050008F7050008F7050008F7050008CF
:10012000F7050008F7050008F7050008F7050008BF
:10013000F7050008F7050008F7050008F7050008AF
:10014000F7050008F7050008F7050008F70500089F
:10015000F7050008F7050008F7050008F70500088F
:10016000F7050008F7050008F7050008F70500087F
:10017000F70500085D540008F7050008F7050008BA
:10018000F7050008F7050008F7050008F70500085F
:10019000F7050008F7050008F7050008F70500084F
:1001A000F7050008F7050008F7050008F70500083F
:1001B000C1600008F7050008F7050008F70500080A
:1001C000F7050008F7050008F7050008F70500081F
:1001D000F705000849540008F7050008F70500086E
:1001E000F7050008F7050008F7050008F7050008FF
:1001F000F7050008F7050008F7050008F7050008EF
:10020000F7050008F7050008F7050008F7050008DE
:10021000F7050008F7050008F7050008F7050008CE
:10022000F7050008F7050008D5480008F70500089D
:10023000F7050008F7050008F7050008F7050008AE
:10024000F7050008F7050008F7050008F70500089E
:10025000F7050008F7050008F7050008F70500088E
:10026000F7050008F7050008F7050008F70500087E
:10027000F7050008F7050008F7050008F70500086E
:10028000F7050008F7050008F7050008F70500085E
:10029000F7050008F7050008F7050008F70500084E
:1002A000F7050008F7050008F7050008F70500083E
:1002B000F7050008F7050008F7050008F70500082E
:1002C000F7050008F7050008F7050008F70500081E
:1002D000F7050008F7050008F7050008F70500080E
:1002E000D9070008091A00082125000800000000AD
:1002F00053B94AB9002908BF00281CBF4FF0FF318D
:100300004FF0FF3000F074B9ADF1080C6DE904CE88
:1003100000F006F8DDF804E0DDE9022304B07047E0
:100320002DE9F047089D04468E46002B4DD18A42A8
:10033000944669D9B2FA82F252B101FA02F3C2F1DB
:10034000200120FA01F10CFA02FC41EA030E94406C
:100350004FEA1C48210CBEFBF8F61FFA8CF708FB8D
:1003600016E341EA034306FB07F199420AD91CEB65
:10037000030306F1FF3080F01F81994240F21C8197
:10038000023E63445B1AA4B2B3FBF8F008FB1033DF
:1003900044EA034400FB07F7A7420AD91CEB040414
:1003A00000F1FF3380F00A81A74240F207816444E4
:1003B000023840EA0640E41B00261DB1D440002369
:1003C000C5E900433146BDE8F0878B4209D9002DCD
:1003D00000F0EF800026C5E9000130463146BDE857
:1003E000F087B3FA83F6002E4AD18B4202D38242C1
:1003F00000F2F980841A61EB030301209E46002D70
:10040000E0D0C5E9004EDDE702B9FFDEB2FA82F2C4
:10041000002A40F09280A1EB0C014FEA1C471FFA22
:100420008CFE0126200CB1FBF7F307FB131140EA09
:1004300001410EFB03F0884208D91CEB010103F1D6
:10044000FF3802D2884200F2CB804346091AA4B298
:10045000B1FBF7F007FB101144EA01440EFB00FE6C
:10046000A64508D91CEB040400F1FF3102D2A645D1
:1004700000F2BB800846A4EB0E0440EA03409CE770
:10048000C6F12007B34022FA07FC4CEA030C20FA1D
:1004900007F401FA06F31C43F9404FEA1C4900FA3D
:1004A00006F3B1FBF9F8200C1FFA8CFE09FB1811BA
:1004B00040EA014108FB0EF0884202FA06F20BD92D
:1004C0001CEB010108F1FF3A80F08880884240F27D
:1004D0008580A8F102086144091AA4B2B1FBF9F0C1
:1004E00009FB101144EA014100FB0EFE8E4508D9BC
:1004F0001CEB010100F1FF346CD28E456AD9023841
:10050000614440EA0840A0FB0294A1EB0E01A14225
:10051000C846A64656D353D05DB1B3EB080261EB93
:100520000E0101FA07F722FA06F3F1401F43C5E96D
:10053000007100263146BDE8F087C2F12003D840A3
:100540000CFA02FC21FA03F3914001434FEA1C47E5
:100550001FFA8CFEB3FBF7F007FB10360B0C43EAD7
:10056000064300FB0EF69E4204FA02F408D91CEB87
:10057000030300F1FF382FD29E422DD90238634485
:100580009B1B89B2B3FBF7F607FB163341EA034125
:1005900006FB0EF38B4208D91CEB010106F1FF3874
:1005A00016D28B4214D9023E6144C91A46EA00466B
:1005B00038E72E46284605E70646E3E61846F8E6FD
:1005C0004B45A9D2B9EB020864EB0C0E0138A3E746
:1005D0004646EAE7204694E74046D1E7D0467BE727
:1005E000023B614432E7304609E76444023842E79F
:1005F000704700BF02E000F000F8FEE772B638482E
:1006000080F30888374880F30988374837490860FD
:1006100040F20000CCF200004EF63471CEF2000140
:100620000860BFF34F8FBFF36F8F40F20000C0F23E
:10063000F0004EF68851CEF200010860BFF34F8FF4
:10064000BFF36F8F4FF00000E1EE100A4EF63C71E1
:10065000CEF200010860062080F31488BFF36F8F8C
:1006600004F02AF904F0CCF805F0B2F94FF0553057
:100670001F491B4A91423CBF41F8040BFAE71D4950
:10068000184A91423CBF41F8040BFAE71A491B4A49
:100690001B4B9A423EBF51F8040B42F8040BF8E79B
:1006A00000201849184A91423CBF41F8040BFAE770
:1006B00004F0E4F805F002FA144C154DAC4203DAEC
:1006C00054F8041B8847F9E700F050F8114C124D1C
:1006D000AC4203DA54F8041B8847F9E704F0CCB8BD
:1006E00000060020002200200000000808ED00E0C5
:1006F0000000002000060020F06800080022002012
:10070000C0220020C0220020904A0020E002000801
:10071000EC020008EC020008EC0200082DE9F04FA2
:100720002DED108AC1F80CD0D0F80CD0BDEC108A99
:10073000BDE8F08F002383F311882846A0470020EE
:1007400003F026FAFEE703F03FF900DFFEE70000C2
:10075000054B10B504460360806810B103685B6800
:100760009847204610BD00BFE064000838B503F08C
:100770006DFF054604F03AF80446F0B9144B9D426B
:100780001DD001339D4241F2883512BF0446002539
:100790000124002003F064FF0CB100F09FF80D4C21
:1007A00000F02EFF00F0C8FD204601F0F1FC40B93A
:1007B00044F6206003F0F2F9F6E70025E9E7054684
:1007C000E7E7284600F046F900F088F8F9E700BFAF
:1007D000010007B0C02200200448054B054A036011
:1007E00000230549836005F0D9BC00BFC02200206A
:1007F000E0640008D42400205107000808B500F088
:1008000067FDA0F120035842584108BD07B50421F7
:1008100001900DEB010000F079FD03B05DF804FBE1
:1008200007B541F21203022101A8ADF8043000F02F
:100830006DFD03B05DF804FB38B5302383F31188F8
:10084000174803680BB103F087FA0023154A4FF4E9
:100850007A71134803F076FA002383F31188124C5F
:10086000236813B12368013B2360636813B1636895
:10087000013B63600D4D2B7833B963687BB902206F
:1008800000F028FE322363602B78032B07D16368C6
:100890002BB9022000F01EFE4FF47A73636038BD5E
:1008A000502300203908000870240020682300200D
:1008B000084B187003280CD8DFE800F00805020880
:1008C000022000F0FFBD022000F0F2BD024B00222A
:1008D0005A6070476823002070240020F7B55648FE
:1008E00001A901F0CDFD002800F0A380534B544A2C
:1008F0001C461968013100F0998004339342F8D105
:100900006268504B9A4240F291804F4BDB6803F192
:10091000104303F580139A4280F08880002000F095
:1009200025FD0220FFF7C4FF484B0021D3F8E82043
:10093000C3F8E810D3F81021C3F81011D3F8102130
:10094000D3F8EC20C3F8EC10D3F81421C3F8141139
:10095000D3F81421D3F8F020C3F8F010D3F81821FD
:10096000C3F81811D3F81821D3F8802042F00062A0
:10097000C3F88020D3F8802022F00062C3F88020E2
:10098000D3F88020D3F8802042F00072C3F8802092
:10099000D3F8802022F00072C3F88020D3F8803092
:1009A00072B64FF0E023C3F8084DD4E90004BFF35A
:1009B0004F8FBFF36F8F264AC2F88410BFF34F8F5B
:1009C000536923F480335361BFF34F8FD2F88030E3
:1009D00043F6E076C3F3C905C3F34E335B0103EA84
:1009E000060C29464CEA81770139C2F87472F9D2B3
:1009F000203B13F1200FF2D1BFF34F8FBFF36F8F66
:100A0000BFF34F8FBFF36F8F536923F400335361EC
:100A10000023C2F85032BFF34F8FBFF36F8F3023E4
:100A200083F31188854680F308882047024801F047
:100A300087F803B0F0BD00BFC02200200000109076
:100A400020001090FFFF0F90002200200044025869
:100A500000ED00E02DE9F04FB34B9FB02022FF21C5
:100A6000089016A89E68DB68079300F073FDAF4AF4
:100A70001378A3B90121AE4811700360302383F3CA
:100A8000118803680BB103F067F90023A94A4FF4FA
:100A90007A71A74803F056F9002383F31188089B65
:100AA00013B1A54B089A1A60A44A1378032B03D0FC
:100AB00000231370A04A53600023089DA04F98465E
:100AC0009B46CDE90533012000F0FCFC25B19A4B93
:100AD0001B68002B00F08783002000F0F9FB0E90CC
:100AE0000E9B002BF2DB012000F0E2FC0E9B213B71
:100AF0001F2BE8D801A252F823F000BF7D0B00089D
:100B0000A50B00083F0C0008C70A0008C70A000828
:100B1000C70A00082B0F000829110008C10F0008A0
:100B2000A7100008CD100008F3100008C70A00083D
:100B300005110008C70A0008711100081D0C000803
:100B4000C70A0008ED110008DD0C0008150E0008AA
:100B5000C70A00081D100008C70A0008C70A0008D5
:100B6000C70A0008C70A0008C70A0008C70A000821
:100B7000C70A0008C70A00083F0C00080220FFF758
:100B80003DFE002840F05B83089B0221069A11A8D5
:100B9000002A08BF1D4641F21233ADF8443000F080
:100BA000B5FB90E74FF47A7000F092FB041EEBDB8C
:100BB0000220FFF723FE0028E6D0013C052C00F2BE
:100BC0004083DFE804F0030A0D10133905230421E4
:100BD00011A8119300F09AFB17E004215248F9E79D
:100BE00004215848F6E704215748F3E74FF01C0961
:100BF000484609F1040900F0BBFB0421119011A83B
:100C000000F084FBB9F12C0FF2D10120059B4FF0CD
:100C1000000B00FA04F41C43E3B2059300F0E6FC79
:100C2000B8F1000F05D0059B03F00B030B2B08BF99
:100C30000025FFF7F5FD46E704214448CAE7B8F16F
:100C4000000FA1D0059B03F00B030B2B9CD10220BE
:100C5000FFF7D4FD0446002896D001204FF000088D
:100C600000F084FB0220FFF723FE5FFA88F9484674
:100C700000F08CFB0546B8B10E99484608F1010812
:100C8000A1F140025142514100F090FB0028ECD10B
:100C90000546069441F21213022111A8A046ADF8B0
:100CA000443000F033FB0EE72E46DFF87C80012055
:100CB000FFF7FEFDD8F80830B34207D9304600F000
:100CC00057FB013040F0C0820436F3E700261B4B8F
:100CD000A04606941E70184B5E609FE7B8F1000FA7
:100CE0003FF452AF059B03F00B030B2B7FF44CAF8B
:100CF00064210FA800F000FB814600287FF444AF78
:100D00000220FFF77BFD044600283FF43DAF3A6A1E
:100D10007B6A0F9953438DF837908B421AD20C4857
:100D200000F0E2FB30E700BF002200206C2400202E
:100D30005023002039080008702400206823002078
:100D4000C022002004220020082200200C220020C3
:100D5000E06200084FF4801AAC48C846BAFBF2FAC9
:100D600000F0C2FBFFF75CFD01210DF1370000F040
:100D7000CDFA0F9B434541D9002310AA514638466E
:100D8000CDE9103311AB00F0DFFE002882D000F077
:100D900099FE109B00EB030901210DF1370000F0D3
:100DA000B5FA00F08FFE484520D9384601F002F927
:100DB00080B964210F9B96480AF1010A01FB08F1F2
:100DC000B1FBF3F18DF83710C9B200F08DFB3B6A2F
:100DD0009844CEE700F076FE119B184448453FF654
:100DE00059AF00F06FFE109B00EB0309109B4FF40E
:100DF0007A70A3FB000302F0D1FECDE7642301214A
:100E00000DF13700A0468DF8373000F07FFA00234F
:100E1000079303E7B8F1000F3FF4B6AE059B03F06C
:100E20000B030B2B7FF4B0AE0220FFF741FD322005
:100E300000F04EFAB0F1000AFFF6A6AE079BD146CD
:100E400053440993734B099ADB689A423FF69CAE70
:100E5000BAF5807F3FF798AE6F4A0024A2450A9208
:100E60000EDD4FF47A7000F033FA0E900E9B002BDB
:100E7000FFF68AAE0E9B01340A9A02F8013BEDE7B9
:100E8000C820FFF7BBFC044600283FF47DAE079B5B
:100E90001F2B11D8C3F1200223F0030016AB5E49CB
:100EA0005245184428BF52460A9200F021FB0A9A84
:100EB000FF21594800F04EFB00239846CDE910333E
:100EC000079B03F580130B93B9F1000F02D1A046E5
:100ED000099B9DE711AB504A0B993846029310AB22
:100EE0004244414401930FAB00934B4601F034FA66
:100EF00000283FF4CFAE00F0E7FD0F9B82460A9139
:100F00009844A9EB030900F0DFFD109B0A9A13EB4C
:100F10000A0342F10002834272EB0103F3D2384626
:100F200001F048F80028EED1CEE7B8F1000F3FF409
:100F30002BAE059B03F00B030B2B7FF425AE022099
:100F4000FFF7B6FC322000F0C3F9B0F1000AFFF65B
:100F50001BAE1AF003047FF417AE2E4A0AEB060309
:100F6000926893423FF610AEBAF5807F3FF70CAE21
:100F7000DFF8A490A2450DDD4FF47A7000F0A8F9D7
:100F80000E900E9B002BFFF6FFAD0E9B013409F86F
:100F9000013BEFE7C820FFF731FC044600283FF48F
:100FA000F3ADCAF387021C4930464FEAAA0900F0A4
:100FB000D9FA804600283FF46DAE06EB89062DE68F
:100FC0000220FFF71BFC00283FF4DEAD00F00CFA16
:100FD00000283FF4D9AD4FF00009DFF838A04C46A7
:100FE000DAF808304B450CD9484609F1040900F0FD
:100FF000BFF90422119011A9204601F0B7FA044666
:10100000EEE72046FFF702FC08E600BF0563000894
:101010001D630008002200206C230020642110A81A
:1010200000F06AF9044600287FF4AEAD0220FFF715
:10103000E5FB00283FF4A8AD109BA14603F0030A8E
:101040001099A1EB0A01A1421BD91F2C11D8169BA4
:1010500001330ED024F003031EAA134453F8203C9E
:1010600011934846042211A9043401F07FFA814605
:10107000E6E7042311AA04F58011384601F0B8F917
:10108000EFE7BAF1000F0CD0534611AA01F5801119
:10109000384601F0ADF94846524611A901F066FA0A
:1010A00081464846AEE70023642111A8119300F061
:1010B00023F900287FF468AD0220FFF79FFB00288A
:1010C0003FF462AD119800F085F99BE7002364219D
:1010D00011A8119300F010F900287FF455AD0220FB
:1010E000FFF78CFB00283FF44FAD119800F074F926
:1010F00088E70220FFF782FB00283FF445AD00F0AF
:1011000083F97FE70220FFF779FB00283FF43CAD2D
:1011100011A9142000F07EF90990FFF777FB0999D7
:1011200011A800F0F3F879E5322000F0D1F8041EA0
:10113000FFF62AADA3077FF427AD444A04EB0B0367
:10114000926893423FF620AD0220FFF757FB00283C
:101150003FF41AAD24F003045C44A3453FF45EADB4
:1011600058460BF1040B00F003F9FFF74FFBF4E7CF
:101170004FF47A70FFF742FB00283FF405AD00F012
:1011800033F980B1169B013328D011AB16AA4FF466
:1011900080113846029310AB01930FAB00932023CC
:1011A00001F0DAF808B9444674E500F08DFC284EE9
:1011B00004460D4600F088FC109B1B1945F1000207
:1011C000834272EB0103F5D2304600F0F3FE0028B3
:1011D000F0D12022FF2116A800F0BCF9FFF720FB78
:1011E0001C4802F0DBFC1FB0BDE8F08FB8F1000F27
:1011F0003FF4CAAC059B03F00B030B2B7FF4C4AC8C
:101200000023642111A8119300F076F80446002809
:101210007FF4BAAC0220FFF7F1FA814600283FF4D0
:10122000B3ACFFF7FDFA41F2883002F0B7FC119839
:1012300000F020FAC846254600F0D8F943E480467D
:10124000ECE44FF0000B9FE4069423E5002200201D
:10125000C0220020A0860100F7B50C46184E4FF4BE
:101260007A71054602FB01F396F90020501C0BD160
:101270001448294601930268176A2246B8478442F7
:10128000019B03D1002310E0002AF1D096F9002041
:10129000511C01D0012A0DD10B4829460268166A5B
:1012A0002246B047844205D10123084A0120137029
:1012B00003B0F0BD4FF4FA7002F070FC0020F7E7C5
:1012C00010220020F82B002000250020BC24002044
:1012D000002307B5024601210DF107008DF8073004
:1012E000FFF7BAFF20B19DF8070003B05DF804FBDB
:1012F0004FF0FF30F9E700000A46042108B5FFF778
:10130000ABFF80F00100C0B2404208BD074B0A4667
:1013100030B41978064B53F8214001462368204623
:10132000DD69044BAC4630BC604700BFBC240020E4
:1013300048630008A086010070B50A4E00240A4DDB
:1013400002F06AFF308028683388834208D902F0AF
:101350005FFF2B6804440133B4F5003F2B60F2D3E8
:1013600070BD00BFBE2400207824002003F008B820
:1013700000F1006000F500300068704700F1006087
:10138000920000F5003002F07FBF0000054B1A68A4
:10139000054B1B889B1A834202D9104402F038BFC8
:1013A0000020704778240020BE24002038B5044671
:1013B000074D29B128682044BDE8384002F034BF09
:1013C0002868204402F02AFF0028F3D038BD00BF6F
:1013D000782400200020704700F1FF5000F58F10A6
:1013E000D0F8000870470000064991F8243033B166
:1013F00000230822086A81F82430FFF7BFBF0120CC
:10140000704700BF7C240020014B1868704700BF64
:101410000010005C244BF0B51A680446234BC2F35D
:101420000B06120C1F885868BE4293F9085028D04A
:101430009F89BE4206D101200C2505FB0033586868
:1014400093F9085041F201039A421CD041F2030380
:101450009A421AD042F201039A4218D042F2030390
:101460009A4208BF5625621E0B46441E0A44934208
:101470000FD214F9016F581C6EB1034600F8016CCD
:10148000F5E70020D8E75A25EDE75925EBE7582581
:10149000E9E7184605E02C2482421C7001D9981C0B
:1014A0005D70401AF0BD00BF0010005C14220020E7
:1014B000022803D1024B4FF400229A61704700BF0B
:1014C00000100258022802D1014B08229A6170478D
:1014D00000100258022804D1024A536983F008031D
:1014E00053617047001002580FB404B070470000F9
:1014F000002310B5934203D0CC5CC4540133F9E708
:1015000010BD0000013810B510F9013F3BB191F951
:1015100000409C4203D11AB10131013AF4E71AB1FB
:1015200091F90020981A10BD1046FCE701380139E6
:1015300010F9013F11F9012F0BB19342F8D0981A1D
:101540007047000003460246D01A12F9011B002919
:10155000FAD1704702440346934202D003F8011BBC
:10156000FAE770472DE9F8431F4D144607468846B1
:1015700095F8242052BBDFF870909CB395F8243086
:101580002BB92022FF2148462F62FFF7E3FF95F891
:1015900024004146C0F1080205EB8000A24228BFAA
:1015A0002246D6B29200FFF7A3FF95F82430A41B81
:1015B00017441E449044E4B2F6B2082E85F8246025
:1015C000DBD1FFF711FF0028D7D108E02B6A03EB2E
:1015D00082038342CFD0FFF707FF0028CBD1002042
:1015E000BDE8F8830120FBE77C240020024B1A7839
:1015F000024B1A70704700BFBC240020102200204C
:1016000038B5164C164D204601F036FC29462046CA
:1016100001F05EFC2D681348D5F89020D2F804380C
:1016200043F00203C2F8043802F0B8FA0E49284623
:1016300001F05CFDD5F890200C48D2F804380C4934
:10164000A04223F00203C2F804384FF4E1330B60E8
:1016500003D0BDE8384001F06DBB38BDF82B002049
:101660003C66000840420F00446600080025002048
:10167000A424002038B50B4B04461A780A4B53F8C3
:1016800022500A4B9D420CD0094B002118221846CB
:10169000FFF760FF046001462846BDE8384001F0CE
:1016A00049BB38BDBC24002048630008F82B00204B
:1016B000A424002038B5084B044615460175436044
:1016C0000A21243003F000F804F128002A460A21F8
:1016D00002F0FAFF204638BD28650008F8B51E461E
:1016E0001B6805460C4617461BB9236863B90124DD
:1016F00008E0BDF818203146806A02F0FDFF00289E
:10170000F3D100242046F8BD21463A46686A03F02A
:1017100029F804460028EAD13368002BF1D0A86AE2
:1017200003F054F8EEE7000038B50D4611460446C4
:101730001A4611B1806A03F007F82DB12946606A94
:10174000BDE8384003F03AB838BD000070470000EB
:1017500070470000002070470020704713B56C46AA
:1017600000F1140384E8060094E8030083E8050010
:1017700002B010BD0020704713B56C4600F10C0399
:1017800084E8060094E8030083E8050002B010BD79
:101790000023C0E90333704782B002AB03E90600BF
:1017A00002B070477047000000207047704700008B
:1017B00000207047002070470120704782B0002051
:1017C00002A901E90C0002B0704700000020704738
:1017D000002070470B6883634B6843638B68C36367
:1017E000CB6803640B6943647047000038B5036B32
:1017F0000446154D1B7955F8330001F073FFD4E909
:101800000B231B7955F8331002F1300349689942D4
:1018100018D000231363E26A5363D4E90B12537C9C
:10182000581E137C92681B0443EA002313438B6306
:10183000D4E90B131B79303155F83300BDE838403B
:1018400001F0E4BE38BD00BFB0630008F8B51D4F1D
:1018500005460E4611463868FFF768FE78BB746887
:101860003B7924B394F82C209A420BD02468F8E7F3
:101870000122B521FFF71EFF736823603B79746076
:1018800084F82C30482004F093FC68B100220271E7
:10189000C0E90322C0E90522027A42F0070202727F
:1018A000094AC0E90B47026028602846F8BD40207D
:1018B00004F07EFC04460028DAD12C60F5E7002312
:1018C0002B60F2E7C0240020C0630008044B10B571
:1018D00004460360406A08B104F068FC204610BD6D
:1018E0006463000810B50446FFF7F0FF204604F0DB
:1018F0005BFC204610BD000008B519B1FFF776FF6C
:10190000012008BD036B1A79024B53F8320001F035
:10191000EDFEF5E7B06300082DE9FF41DDF8288012
:101920000546174603911FFA88F60293FFF75EFFFC
:1019300002ABBAB203A9E86A0096FFF7CFFE0446ED
:1019400038B900212846FFF7D7FF204604B0BDE88C
:10195000F081AFB92B6B05F134011A79134B53F8B1
:101960003200B8F1000F19D101F05EFE80F00104E1
:10197000E4B23346E86ADDE90221FFF7D5FEE0E78D
:10198000029B83B92B6B3A46084805F134011C7958
:10199000039B50F8340001F05DFEE7E7029B4246EE
:1019A00001F06EFEE2E70024E3E700BFB063000849
:1019B00013B504460191FFF719FF019A236B04F157
:1019C00034011879054B53F8300001F06FFE002107
:1019D0002046FFF791FF012002B010BDB063000860
:1019E00010B50446FFF702FF236B1A79054B53F835
:1019F000320001F069FE00212046FFF77DFF012043
:101A000010BD00BFB0630008064B0121064A1A60F2
:101A100000221A71054AC3E902124FF48C721A822D
:101A2000704700BFC02400205063000800E1F505A6
:101A300000B59BB0EFF3098168226846FFF758FDB7
:101A4000EFF30583044B9A6BDA6A9A6A9A6A9A6A88
:101A50009A6A9A6A9B6AFEE700ED00E000B59BB0C7
:101A6000EFF3098168226846FFF742FDEFF3058333
:101A7000044B9A6B9A6A9A6A9A6A9A6A9A6A9B6AF9
:101A8000FEE700BF00ED00E000B59BB0EFF3098179
:101A900068226846FFF72CFDEFF30583034B5A6B72
:101AA0009A6A9A6A9A6A9A6A9B6AFEE700ED00E06F
:101AB000FEE70000FEE700000FB408B5029801F051
:101AC000F9FFFEE702F062BD02F03ABD806970479F
:101AD000C0697047006A7047406A7047806A704703
:101AE000F0B5ADF2044D0E46054600214FF47F726D
:101AF00001A80091FFF72EFD2C6A744301362B6A72
:101B00007343A34216D92B686A46214628465F686C
:101B10004FF48063B84770B16A464FF4806312F89F
:101B2000011BFF290AD1013B9BB2002BF7D104F521
:101B30008064E4E701200DF2044DF0BD0020FAE7D7
:101B400080680368DB69184730B5456A85B004468C
:101B50008D420FD30568CDE90023026A03ABAD6A5D
:101B60005143A84720B1206A039BC31A58425841E9
:101B700005B030BD0020FBE7F0B5C56987B004466D
:101B80008D4212D30C9F866905687143CDE90137F8
:101B900005AB00936D69036AA84720B1A069059B56
:101BA000C31A5842584107B0F0BD0020FBE70000BF
:101BB000F0B5662389B0002405464FF4807680682E
:101BC000079403A9CDE90336CDE9054403685B69B1
:101BD0009847A86822462146036800941F69234657
:101BE000B847A8689923079403A9CDE90336CDE93E
:101BF000054403685B699847A86822462146036844
:101C000000941D692346A84709B0F0BD254B2DE976
:101C1000F04F1B789FB0002504468DF828304FF018
:101C20009F0E80684FF00123ADF8295005A9099552
:101C3000CDE905E3CDE9075503685B699847A068DE
:101C400003222946036800922A461E690AABB04760
:101C500028B394F88C20144B9DF8281003EBC20392
:101C60001A7991421BD19DF829205B799A4216D1AD
:101C7000A0684FF05A0C0D4B082605A90996CDE92E
:101C800005C3CDE9075503685B699847A0682A46F4
:101C90002946036800961F690AABB84740B900207F
:101CA00048E100BFC8620008C064000800250001C8
:101CB0000422B1490AA804F0ABFA05460028EED187
:101CC000BDF82C306FF48277A3813B44012BE6D81A
:101CD000079605A9CDE90A00A06803685B699847E3
:101CE000A0682A462946036800961E690AABB047D9
:101CF0000028D4D0DDE90A361A0202F4706242EA02
:101D00001662FF2ACBD11B0E26F07F4650222946B1
:101D1000142B26610AA828BF1423A373FFF71AFC0B
:101D2000A068079605A903685B699847A068A37B2C
:101D3000294602689B0000930AAB16692A46B04701
:101D40000028ACD00B990029A9DBC9086FF07E43AD
:101D5000149D4FF0010E994228BF1946C5F3031395
:101D60000EFA03F221FA03F303916161A261E361C8
:101D7000002B94D02646A44600274FF002081EAA46
:101D8000C7F3460302EB830353F834AC07F00103B7
:101D90001B01DA1D0EFA03F908FA02F2A2EB09029E
:101DA00002EA0A02DA401AD003F108090F330EFAE8
:101DB00002F2216A08FA03F30EFA09FBCCF830208C
:101DC0008A42A3EB0B0B0BEA0A0A2AFA09F98CF8F0
:101DD0002C90A36A88BF2262934288BFA262013717
:101DE0000CF1100C042FCAD1236A4FF0020C039A95
:101DF0004FF0010E139F9A4224BFB2FBF3F16162D0
:101E000007F00F0138BF01234FF0090201F1010172
:101E100038BF63624900336B33B3531C0EFA02F8C8
:101E2000A2F105090CFA03F30EFA09FAA3EB080371
:101E300002F1FF380CFA08F83B40A8EB0A08D3403F
:101E400008EA070828FA09F877D0012B77D0022B87
:101E500077D0032B08BF4FF47A735FFA88F808FB3A
:101E6000033373634B43B36307321036252AD2D151
:101E700015F0C04FC5F3417365D0012B65D0022B1F
:101E80000CBF4FF47A634FF47A43C5F3046202FB4C
:101E90000333E3664B432367199B9E0758D0062301
:101EA00084F8743015F4005F05F00F03C5F30425C2
:101EB00014BF40220822013305FB02255B00A56701
:101EC0005D430A9B9F02E5677FF5E9AE0C9B1A0A0A
:101ED00084F88020C3F3421203F01F0384F88820A3
:101EE00084F88130189BC3F3025213F4401F84F826
:101EF00083207FF4D4AEDE0602D5042A7FF4CFAE71
:101F000003F40072002A14BF0122002284F8872003
:101F100004D0DD0324D5002384F88930179B1A07E9
:101F200022D5002384F88630702384F8853001237D
:101F300084F88D301FB0BDE8F08F01238DE71023AA
:101F40008BE7802389E710239FE74FF480739CE79A
:101F5000590701D55023A3E713F0780FA2D09EE6CE
:101F60009903DBD50123D7E75B07E0D5012384F88C
:101F700086300523D9E700BF2064000830B58BB058
:101F800000240546806803924FF00122059105A9BF
:101F9000CDE90624CDE90844026852699047A86853
:101FA0000121039B02680091214615692246A8473A
:101FB0000BB030BD13B504460DF1070290F8851043
:101FC000FFF7DCFF94F886309DF807001BB100F0A6
:101FD000010002B010BDC043C0F3C010F9E700001B
:101FE00030B54FF001238BB00024054680688DF892
:101FF0000F20059105A9CDE90634CDE90844036811
:102000005B699847A86801220DF10F0103680094ED
:102010001D692346A8470BB030BD0000F7B5174631
:102020000DF1070206461D46FFF7A8FF68B19DF8AF
:10203000074039469DF82020304624EA05042A400E
:1020400022438DF80720FFF7CBFF03B0F0BD00005F
:1020500030B54FF4807389B0002405468068039141
:1020600003A9CDE90434CDE9064403685B699847C8
:10207000A86822462146036800941D692346A847A4
:1020800009B030BD10B5044623682046DB6A984786
:102090000028F9D110BD000010B590F87430044646
:1020A0005BB1FFF7EFFF012394F87410204684F82A
:1020B0008E30BDE81040FFF7CBBF012010BD0000FF
:1020C00010B590F87430044653B1FFF7DBFF0123DD
:1020D0002046042184F88E30BDE81040FFF7B8BFD9
:1020E000012010BD70B590F883308AB00446042BEF
:1020F00048D10DF10E020521FFF740FF00282FD037
:102100000DF10F0235212046FFF738FF40B320467E
:102110001E4EFFF7C1FF2046FFF7B4FF05AD0FCEFF
:102120000FC5336805A99DF80E202B609DF80F3070
:10213000A06843F002038DF810208DF80F308DF861
:10214000113003685B699847A068002304A90268FE
:10215000009315690222A84728B92046FFF7B0FF6F
:1021600000200AB070BD2046FFF7AAFF0DF10F0254
:1021700035212046FFF702FF0028F1D09DF80F30EF
:102180009B07EDD501202071EBE700BFCC62000872
:102190002DE9F341002304468068A36010B1036871
:1021A0005B6898470025244E244F56F8352001A837
:1021B00039465FFA85F8FFF749FB019BA0680022CA
:1021C000A360019210B103685B689847019810B151
:1021D00003685B689847A368DBB141F2883084F8F4
:1021E0008C8001F0DBFC2046FFF7E2FC1E2001F0B2
:1021F000D5FC2046FFF70AFD054680B994F88C30DF
:102200000F4856F83310FFF76FF9284602B0BDE8C3
:10221000F0810135032DC8D10A48FFF74DFC204657
:10222000FFF760FF94F88C30054656F8331008B974
:102230000548E8E70548E6E7C0640008D824002020
:10224000286400089E640008526400087C6400084A
:102250002DE9F041044688B00F461646FFF71CFFF3
:102260002046FFF70FFF0025C722A0684FF48073B8
:10227000079503A9CDE90323CDE9055503685B69FB
:102280009847A0682A46294603680095D3F810802D
:102290002B46C047054630B92046FFF711FF2846B8
:1022A00008B0BDE8F081E36E3B60236F3360F3E775
:1022B0002DE9F041002588B01F4604460E460E9BCE
:1022C00000F1400CA8463D60016B81B1A9420ED3DC
:1022D00091420CD8B6FBF1FE01FB1E6139B9416B8E
:1022E00090F82C800F9D1960816B29601546103085
:1022F0006045E9D16DB3AB196269934229D8204694
:10230000FFF7CAFE2046FFF7BDFE4FF41453A06846
:1023100003A9CDF80C80CDE904360026CDE9066688
:1023200003685B699847A0683246314603680096A7
:10233000D3F810803346C047064620462EB9FFF733
:10234000BFFE304608B0BDE8F081FFF7B9FE3D6042
:10235000F7E70026F5E700002DE9F041866905461C
:1023600088B00F46B3429046B1FBF6FC06FB1C1C3E
:1023700028BF3346A6EB0C0C00269C45644628BFBC
:102380001C46FFF789FE2846FFF77CFE0222A8685C
:1023900003A9164B0597CDE90323CDE9066603682B
:1023A0005B699847A86822464146036800961F6902
:1023B0003346B847064628462EB9FFF781FE304619
:1023C00008B0BDE8F081FFF77BFE0E9B1C60AB6F91
:1023D000AA696343B3FBF2F30F9A1360EA6F109B91
:1023E0005443AA69B4FBF2F41C60E8E7002500013D
:1023F0002DE9F04FCE18436989B004469E420F463E
:10240000904634D83D464FF00009DFF870A0FFF742
:1024100039FEAE422FD9A6EB050B94F8803094F824
:10242000882003A9BBF5806F039394F8813028BFFF
:102430004FF4806B012AA06808BF03F1FF33CDF889
:1024400010A0CDE90559079303685B699847A06818
:10245000A8EB07030268CDF800B02B44D2F810B007
:1024600000221146D84718B105F58065D1E7002054
:1024700009B0BDE8F08F0120FAE700BF00ED0003CE
:10248000F0B5044689B00E46FFF7FCFD94F887507E
:102490002DB194F889302BB1012B1DD00025284691
:1024A00009B0F0BD94F880200392F02206921A4AF7
:1024B000CDE9042394F88130A06803A90793036849
:1024C0005B699847A068314603689B699847054651
:1024D000642001F063FBE2E720460027FFF7DCFD04
:1024E0002046FFF7CFFD0823812285212046009753
:1024F000FFF794FD054618B92046FFF7E1FDCEE74A
:1025000094F8803006970393044BCDE9043794F890
:102510008130013BD0E700BF00ED000300ED001368
:10252000014B024A1A607047D82400201464000846
:10253000036800211B68184703790BB10022027160
:102540001846704703685B681847000003791BB999
:102550000123037118467047002070477047000040
:1025600010B5044603F020FE204610BD30B50A44E5
:10257000084D91420DD011F8013B5840082340F31B
:102580000004013B2C4013F0FF0384EA5000F6D115
:10259000EFE730BD2083B8ED8A0710B504461DD59E
:1025A0000378042B1AD143681B682BB105220270F3
:1025B00098472378052B01D102232370302383F31E
:1025C0001188002104F1080001F002FB002383F3CD
:1025D0001188E069BDE8104002F040BACB0704D58D
:1025E0000248BDE8104001F065BA10BD4065000822
:1025F00010B5044C204601F001F8034A0023C4E959
:10260000062310BDE02400200050005210B50378CE
:102610000446012B17D1104B984214D102460F49A2
:10262000102002F0E7F90E4BE061D3F8D42042F419
:102630008042C3F8D420D3F8FC2042F48042C3F88F
:10264000FC20D3F8FC306268A36992685A60054A9E
:102650001A601B22DA6010BDE024002099250008D2
:10266000004402581500020182691B2310B5D36093
:10267000D1E9003013F44C4406D19B011461D061C0
:1026800003F44043536110BD0024184313F4406F1A
:102690001461CC68D4615061F5D08B689361F2E726
:1026A00030B584691B25C069E5600068836104F169
:1026B0002003C36102234261013A03614223C360E4
:1026C00016238362CB682261E361D1E900231343BF
:1026D00012F4406F636101D08B68A361C36843F05B
:1026E0000103C36030BD000030B5D0E9064000688A
:1026F00004F120058561C36108234261013A036149
:1027000046230D69C36016238362CB682261E361AF
:10271000D1E90023134312F4406F43EA854343F0A9
:102720008063636101D08B68A361C36843F00103D8
:10273000C36030BD8069036823F0040310B5CC6822
:10274000036000230361C4618361D1E90043096927
:10275000234343EA814343F04063436112B14FF0A6
:102760001043136010BD000083691A6842F0020232
:102770001A601A689207FCD41A6842F004021A60C0
:10278000704700008269936810B5D3609B070446C8
:102790001DD50378032B1AD143681B682BB1052282
:1027A000027098472378052B01D102232370302330
:1027B00083F31188002104F1080001F009FA0023D5
:1027C00083F31188E069BDE8104002F047B910BDFD
:1027D000026843681143016003B118477047000065
:1027E000024A136843F0C0031360704700100140B1
:1027F00013B50E4C204600F091FA04F114000023AA
:102800004FF400720A49009400F04EF9094B4FF45E
:102810000072094904F13800009400F0C7F9074A32
:10282000074BC4E9172302B010BD00BF00250020EC
:102830006C250020E12700086C27002000100140D3
:1028400000E1F505037C30B5244C002918BF0C4687
:10285000012B11D1224B98420ED1224BD3F8F020FC
:1028600042F01002C3F8F020D3F8182142F0100211
:10287000C3F81821D3F818312268036EC16D03EB39
:1028800052038466B3FBF2F36268150442BF23F07F
:10289000070503F0070343EA4503CB60A36843F051
:1028A00040034B60E36843F001038B6042F496738E
:1028B00043F001030B604FF0FF330B62510505D568
:1028C00012F0102205D0B2F1805F04D080F864309D
:1028D00030BD7F23FAE73F23F8E700BF50650008CB
:1028E00000250020004402582DE9F047C66D05463A
:1028F0003768F469210734621AD014F0080118BF50
:102900004FF48071E20748BF41F02001A3074FF068
:10291000300348BF41F04001600748BF41F08001EB
:1029200083F31188281DFFF753FF002383F31188D9
:10293000E2050AD5302383F311884FF48061281D06
:10294000FFF746FF002383F311884FF030094FF063
:10295000000A14F0200838D13B0616D54FF0300994
:1029600005F1380A200610D589F31188504600F089
:1029700051F9002836DA0821281DFFF729FF27F032
:1029800080033360002383F31188790614D562062F
:1029900012D5302383F31188D5E913239A4208D145
:1029A0002B6C33B127F040071021281DFFF710FFD3
:1029B0003760002383F31188E30618D5AA6E1369E4
:1029C000ABB15069BDE8F047184789F31188736AC5
:1029D000284695F86410194000F0BAF98AF3118876
:1029E000F469B6E7B06288F31188F469BAE7BDE824
:1029F000F0870000F8B51546826804460B46AA42E7
:102A000000D28568A1692669761AB5420BD21846AC
:102A10002A46FEF76DFDA3692B44A3612846A368EF
:102A20005B1BA360F8BD0CD9AF1B18463246FEF7FE
:102A30005FFD3A46E1683044FEF75AFDE3683B44E7
:102A4000EBE718462A46FEF753FDE368E5E700008A
:102A500083689342F7B50446154600D28568D4E9E9
:102A60000460361AB5420BD22A46FEF741FD63696F
:102A70002B4463612846A3685B1BA36003B0F0BDD1
:102A80000DD93246AF1B0191FEF732FD01993A464E
:102A9000E0683144FEF72CFDE3683B44E9E72A4651
:102AA000FEF726FDE368E4E710B50A440024C3619D
:102AB000029B8460C16002610362C0E90000C0E95A
:102AC000051110BD08B5D0E90532934201D18268E5
:102AD00082B98268013282605A1C426119700021F9
:102AE000D0E904329A4224BFC368436101F08AF8F6
:102AF000002008BD4FF0FF30FBE7000070B5302329
:102B000004460E4683F31188A568A5B1A368A2699F
:102B1000013BA360531CA36115782269934224BF33
:102B2000E368A361E3690BB120469847002383F370
:102B30001188284607E03146204601F053F8002866
:102B4000E2DA85F3118870BD2DE9F74F04460E4691
:102B500017469846D0F81C904FF0300A8AF3118837
:102B60004FF0000B154665B12A4631462046FFF767
:102B700041FF034660B94146204601F033F8002882
:102B8000F1D0002383F31188781B03B0BDE8F08FE8
:102B9000B9F1000F03D001902046C847019B8BF389
:102BA0001188ED1A1E448AF31188DCE7C160C36105
:102BB000009B82600362C0E905111144C0E9000076
:102BC00001617047F8B504460D461646302383F37D
:102BD0001188A768A7B1A368013BA36063695A1C69
:102BE00062611D70D4E904329A4224BFE3686361D4
:102BF000E3690BB120469847002080F3118807E075
:102C00003146204600F0EEFF0028E2DA87F3118813
:102C1000F8BD0000D0E9052310B59A4201D18268C1
:102C20007AB982680021013282605A1C82611C7864
:102C300003699A4224BFC368836100F0E3FF204622
:102C400010BD4FF0FF30FBE72DE9F74F04460E466D
:102C500017469846D0F81C904FF0300A8AF3118836
:102C60004FF0000B154665B12A4631462046FFF766
:102C7000EFFE034660B94146204600F0B3FF00284E
:102C8000F1D0002383F31188781B03B0BDE8F08FE7
:102C9000B9F1000F03D001902046C847019B8BF388
:102CA0001188ED1A1E448AF31188DCE70268436834
:102CB0001143016003B11847704700001430FFF75B
:102CC00043BF00004FF0FF331430FFF73DBF00005B
:102CD0003830FFF7B9BF00004FF0FF333830FFF74F
:102CE000B3BF00001430FFF709BF00004FF0FF3101
:102CF0001430FFF703BF00003830FFF763BF000058
:102D00004FF0FF323830FFF75DBF0000012914BFDC
:102D10006FF0130000207047FFF76ABD044B03609B
:102D200000234360C0E9023301230374704700BFEE
:102D30006865000810B53023044683F31188FFF757
:102D400081FD02230020237480F3118810BD000050
:102D500038B5C36904460D461BB904210844FFF782
:102D6000A5FF294604F11400FFF7ACFE002806DA9F
:102D7000201D4FF40061BDE83840FFF797BF38BD14
:102D8000026843681143016003B1184770470000AF
:102D900013B5406B00F58054D4F8A4381A68117844
:102DA000042914D1017C022911D119790123128936
:102DB0008B4013420BD101A94C3002F097FCD4F8A0
:102DC000A4480246019B2179206800F0DFF902B097
:102DD00010BD0000143002F019BC00004FF0FF33AA
:102DE000143002F013BC00004C3002F0EBBC0000C9
:102DF0004FF0FF334C3002F0E5BC0000143002F01D
:102E0000E7BB00004FF0FF31143002F0E1BB0000DF
:102E10004C3002F0B7BC00004FF0FF324C3002F0F3
:102E2000B1BC00000020704710B500F58054D4F804
:102E3000A4381A681178042917D1017C022914D109
:102E40005979012352898B4013420ED1143002F07C
:102E500079FB024648B1D4F8A4484FF44073617935
:102E60002068BDE8104000F07FB910BD406BFFF74F
:102E7000DBBF0000704700007FB5124B0125042620
:102E8000044603600023057400F184024360294670
:102E9000C0E902330C4B0290143001934FF440739D
:102EA000009602F02BFB094B04F69442294604F1EC
:102EB0004C000294CDE900634FF4407302F0F2FB42
:102EC00004B070BD906500086D2E0008912D0008BB
:102ED0000A68302383F311880B790B3342F82300FF
:102EE0004B79133342F823008B7913B10B3342F83B
:102EF000230000F58053C3F8A418022303740020B4
:102F000080F311887047000038B5037F044613B181
:102F100090F85430ABB90125201D0221FFF730FF96
:102F200004F114006FF00101257700F077FE04F141
:102F30004C0084F854506FF00101BDE8384000F0B7
:102F40006DBE38BD10B5012104460430FFF718FFEF
:102F50000023237784F8543010BD000038B50446B0
:102F60000025143002F0E2FA04F14C00257702F05B
:102F7000B1FB201D84F854500121FFF701FF2046CA
:102F8000BDE83840FFF750BF90F8803003F0600391
:102F9000202B06D190F881200023212A03D81F2A54
:102FA00006D800207047222AFBD1C0E91D3303E078
:102FB000034A426707228267C3670120704700BF48
:102FC0002C22002037B500F58055D5F8A4381A68B2
:102FD000117804291AD1017C022917D1197901230A
:102FE00012898B40134211D100F14C04204602F0AB
:102FF00031FC58B101A9204602F078FBD5F8A4486D
:103000000246019B2179206800F0C0F803B030BD72
:1030100001F10B03F0B550F8236085B004460D466E
:10302000FEB1302383F3118804EB8507301D08219E
:10303000FFF7A6FEFB6806F14C005B691B681BB13D
:10304000019002F061FB019803A902F04FFB0246D8
:1030500048B1039B2946204600F098F8002383F3EB
:10306000118805B0F0BDFB685A691268002AF5D0D6
:103070001B8A013B1340F1D104F18002EAE7000012
:10308000133138B550F82140ECB1302383F3118867
:1030900004F58053D3F8A4281368527903EB820314
:1030A000DB689B695D6845B104216018FFF768FE25
:1030B000294604F1140002F04FFA2046FFF7B4FE4F
:1030C000002383F3118838BD7047000001F01CBD58
:1030D00001234022002110B5044600F8303BFEF7E2
:1030E00039FA0023C4E9013310BD000010B53023C4
:1030F000044683F311882422416000210C30FEF73E
:1031000029FA204601F022FD02230020237080F3DB
:10311000118810BD70B500EB8103054650690E465D
:103120001446DA6018B110220021FEF713FAA069E4
:1031300018B110220021FEF70DFA31462846BDE8ED
:10314000704001F009BE000083682022002103F0D6
:10315000011310B5044683601030FEF7FBF92046DA
:10316000BDE8104001F084BEF0B4012500EB8104FD
:1031700047898D40E4683D43A4694581236000236D
:10318000A2606360F0BC01F0A1BE0000F0B40125B4
:1031900000EB810407898D40E4683D436469058143
:1031A00023600023A2606360F0BC01F017BF000041
:1031B00070B5022300250446242203702946C0F876
:1031C00088500C3040F8045CFEF7C4F9204684F8BF
:1031D000705001F055FD63681B6823B129462046F5
:1031E000BDE87040184770BD037880F88C30052327
:1031F000037043681B6810B504460BB1042198475F
:103200000023A36010BD000090F88C20436802707A
:103210001B680BB1052118477047000070B590F886
:103220007030044613B1002380F8703004F180023E
:10323000204601F041FE63689B68B3B994F8803082
:1032400013F0600535D00021204602F01DF9002161
:10325000204602F00DF963681B6813B10621204671
:103260009847062384F8703070BD204698470028A0
:10327000E4D0B4F88630A26F9A4288BFA36794F96D
:103280008030A56F002B4FF0300380F20381002DBA
:1032900000F0F280092284F8702083F31188002165
:1032A0002046D4E91D23FFF771FF002383F3118823
:1032B000DAE794F8812003F07F0343EA022340F227
:1032C0000232934200F0C58021D8B3F5807F48D008
:1032D0000DD8012B3FD0022B00F09380002BB2D1F0
:1032E00004F1880262670222A267E367C1E7B3F5CF
:1032F000817F00F09B80B3F5407FA4D194F88230A9
:10330000012BA0D1B4F8883043F0020332E0B3F5CA
:10331000006F4DD017D8B3F5A06F31D0A3F5C063BF
:10332000012B90D86368204694F882205E6894F858
:103330008310B4F88430B047002884D043686367B2
:103340000368A3671AE0B3F5106F36D040F6024267
:1033500093427FF478AF5C4B63670223A36700233B
:10336000C3E794F88230012B7FF46DAFB4F8883056
:1033700023F00203A4F88830C4E91D55E56778E717
:10338000B4F88030B3F5A06F0ED194F882302046A7
:1033900084F88A3001F0D2FC63681B6813B1012104
:1033A00020469847032323700023C4E91D339CE77C
:1033B00004F18B0363670123C3E72378042B10D147
:1033C000302383F311882046FFF7BEFE85F3118872
:1033D0000321636884F88B5021701B680BB1204671
:1033E000984794F88230002BDED084F88B30042389
:1033F000237063681B68002BD6D0022120469847B3
:10340000D2E794F8843020461D0603F00F010AD558
:1034100001F044FD012804D002287FF414AF2B4BA7
:103420009AE72B4B98E701F02BFDF3E794F88230F5
:10343000002B7FF408AF94F8843013F00F01B3D061
:103440001A06204602D502F037F8ADE702F028F858
:10345000AAE794F88230002B7FF4F5AE94F884301C
:1034600013F00F01A0D01B06204602D502F00CF885
:103470009AE701F0FDFF97E7142284F8702083F3A8
:1034800011882B462A4629462046FFF76DFE85F314
:103490001188E9E65DB1152284F8702083F3118864
:1034A00000212046D4E91D23FFF75EFEFDE60B2236
:1034B00084F8702083F311882B462A46294620463B
:1034C000FFF764FEE3E700BFC0650008B8650008C9
:1034D000BC65000838B590F870300446002B3ED02B
:1034E000063BDAB20F2A34D80F2B32D8DFE803F0CC
:1034F00037313108223231313131313131313737E1
:10350000856FB0F886309D4214D2C3681B8AB5FB24
:10351000F3F203FB12556DB9302383F311882B4668
:103520002A462946FFF732FE85F311880A2384F8DC
:1035300070300EE0142384F87030302383F3118848
:10354000002320461A461946FFF70EFE002383F398
:10355000118838BDC36F03B198470023E7E7002106
:10356000204601F091FF0021204601F081FF6368B1
:103570001B6813B10621204698470623D7E70000B1
:1035800010B590F870300446142B29D017D8062BAC
:1035900005D001D81BB110BD093B022BFBD800217F
:1035A000204601F071FF0021204601F061FF6368B1
:1035B0001B6813B1062120469847062319E0152BF6
:1035C000E9D10B2380F87030302383F31188002376
:1035D0001A461946FFF7DAFD002383F31188DAE76C
:1035E000C3689B695B68002BD5D1C36F03B1984753
:1035F000002384F87030CEE7FEF7FABF01210023E4
:103600000170C0E901330C3000F0FEB910B5302371
:10361000044683F311884160FEF7F8FF022300207F
:10362000237080F3118810BD10B53023044683F356
:103630001188032304F8083BFFF716F84FF0FF3119
:10364000204600F0B7FA002383F31188C01A18BF90
:10365000012010BD38B50446302585F311880325B7
:1036600004F8085BFFF71CF84FF0FF31204600F02C
:10367000A1FA002383F31188C01A18BF012038BDB6
:1036800038B50446302585F31188042504F8085B15
:10369000FFF72AF84FF0FF31204600F08BFA0023A5
:1036A00083F31188C01A18BF012038BD10B530232C
:1036B000044683F31188FFF73DF8062323700023A7
:1036C00083F3118810BD000010B53023044683F346
:1036D0001188FFF749F802232370002383F3118830
:1036E00010BD00000C3000F0ABB900000C3000F051
:1036F000B1B9000004480121044B03600023C0E974
:1037000001330C3000F080B96C2900200959000801
:10371000CB1D083A23F00703591A521A012110B49D
:10372000D2080024C0E9004384600C301C605A6059
:103730005DF8044B00F068B92DE9F84F364ECD1D09
:103740000F46002818BF0646082A4FEAD50538BF9D
:10375000082206F10C08341D9146404600F070F92D
:1037600009F10701C9F1000E224624686CB94046F0
:1037700000F070F93368CBB308224946E800984757
:10378000044698B340E9026730E004EB010CD4F83A
:1037900004A00CEA0E0C0AF10100ACF1080304EBE2
:1037A000C0009842E0D9A0EB0C0CB5EBEC0F4FEA4F
:1037B000EC0BD9D89C421CD204F10802AB45A3EB18
:1037C00002024FEAE202626009D9691CED432068F7
:1037D00003EBC1025D44556043F8310022601C4692
:1037E0005F60404644F8086B00F034F92046BDE8BD
:1037F000F88FAA45216802D111602346EFE7013511
:1038000004EBC50344F8351003F10801401AC01059
:1038100058601360F1E700BF6C290020F8B550F83C
:10382000043C044650F8085CA0F1080607332F1D3D
:103830000C35DB0840F8043C284600F001F93B4613
:103840009F421A6801D0B34228D20AB1964225D2CB
:1038500044F8082C54F8042C1E60013254F8081C5B
:1038600006EBC200814206D14868024444F8042CA9
:103870000A6844F8082C5868411C03EBC1018E42C9
:1038800007D154F8042C013202445A6054F8082C31
:103890001A602846BDE8F84000F0DCB81346CFE7D0
:1038A00000238268037503691B6899689142FBD203
:1038B0005A68036042601060586070470023826855
:1038C000037503691B6899689142FBD85A680360C5
:1038D000426010605860704708B50846302383F393
:1038E00011880A7D0023052A06D8DFE802F00B05BF
:1038F0000503120E826913604FF0FF338361FFF7F7
:10390000CFFF002383F3118808BD826993680133D8
:103910009360D0E9003213605A60EDE7FFF7C0BF53
:10392000054BD96808751868026853601A6001224F
:10393000D8600275FCF7F2BE882900200C4B30B528
:10394000DD684B1C87B004460FD02B46094A6846F9
:1039500000F0F8F92046FFF7E3FF009B13B168463B
:1039600000F0FAF9A86907B030BDFFF7D9FFF9E711
:1039700088290020D938000838B50C4D04468161EB
:10398000EB6881689A68914203D8BDE83840FFF738
:1039900087BF1846FFF792FF01230146EC602046DF
:1039A0002375BDE83840FCF7B9BE00BF8829002068
:1039B000044B1A68DB6890689B68984294BF0020AB
:1039C0000120704788290020084B10B51C68D86872
:1039D000226853601A600122DC602275FFF76EFFD7
:1039E00001462046BDE81040FCF798BE882900201B
:1039F000044B1A68DB6892689B689A4201D9FFF70A
:103A0000E3BF704788290020C0E90000816070474B
:103A10008368013B002B10B583600CDA074BDC6830
:103A20004368A061206063601C6044600520FFF76C
:103A300077FFA06910BD0020FCE700BF88290020A7
:103A400008B5302383F31188FFF7E2FF002383F3E7
:103A5000118808BD08B5302383F3118883680133CA
:103A6000002B836007DC036800211A680260506045
:103A70001846FFF781FF002383F3118808BD00007B
:103A800038B50123084C00252370656001F01EFF46
:103A9000FFF730FE0549064801F042FF022323707C
:103AA00085F3118838BD00BFF02B0020C8650008E1
:103AB0008829002008B572B6044B186500F032FD65
:103AC00000F000FE024B03221A70FEE78829002056
:103AD000F02B002000F076B9EFF3118020B9EFF35E
:103AE0000583302282F311887047000010B530B989
:103AF000EFF30584C4F3080414B180F3118810BDFA
:103B0000FFF776FF84F31188F9E70000034A516854
:103B100053685B1A9842FBD8704700BF001000E062
:103B20008B600223086108468B8270478368A3F18B
:103B3000840243F8142C026943F8442C426943F888
:103B4000402C094A43F8242CC268A3F1200043F812
:103B5000182C022203F80C2C002203F80B2C034A29
:103B600043F8102C704700BF350700088829002053
:103B700008B5FFF7DBFFBDE80840FFF7CFBE000048
:103B8000024BDB6898610F20FFF7CABE882900202E
:103B9000302383F31188FFF7F3BF000008B5014617
:103BA000302383F311880820FFF7C8FE002383F336
:103BB000118808BD054BDB6821B1036098610320C3
:103BC000FFF7BCBE4FF0FF30704700BF88290020D0
:103BD00003682BB10022026018469961FFF79EBE70
:103BE00070470000064BDB6839B1426818605A60C4
:103BF000136043600420FFF7A1BE4FF0FF30704711
:103C0000882900200368984206D01A680260506034
:103C100018469961FFF782BE7047000038B5044628
:103C20000D462068844200D138BD036823605C6083
:103C30008561FFF773FEF4E7036810B59C68A24244
:103C40000CD85C688A600B604C6021605960996890
:103C50008A1A9A604FF0FF33836010BD121B1B68F5
:103C6000ECE700000A2938BF0A2170B504460D466A
:103C70000A26601901F024FE01F00CFE041BA54287
:103C800003D8751C04462E46F3E70A2E04D90120FA
:103C9000BDE8704001F084BE70BD0000F8B5144B63
:103CA0000D460A2A4FF00A07D96103F1100182601C
:103CB00038BF0A22416019691446016048601861E2
:103CC000A81801F0EDFD01F0E5FD431B0646A342F7
:103CD00006D37C1C28192746354601F0F1FDF2E792
:103CE0000A2F04D90120BDE8F84001F059BEF8BD03
:103CF00088290020F8B506460D4601F0CBFD0F4A95
:103D0000134653F8107F9F4206D12A46014630469B
:103D1000BDE8F840FFF7C2BFD169BB68441A2C194F
:103D200028BF2C46A34202D92946FFF79BFF224613
:103D300031460348BDE8F840FFF77EBF88290020E0
:103D400098290020C0E90323002310B45DF8044B38
:103D50004361FFF7CFBF000010B5194C23699842AB
:103D60000DD08168D0E9003213605A609A680A4425
:103D70009A60002303604FF0FF33A36110BD026817
:103D8000234643F8102F53600022026022699A42B2
:103D900003D1BDE8104001F08DBD936881680B44EC
:103DA000936001F077FD2269E1699268441AA242AA
:103DB000E4D91144BDE81040091AFFF753BF00BF12
:103DC000882900202DE9F047DFF8BC8008F11007B2
:103DD0002C4ED8F8105001F05DFDD8F81C40AA68B0
:103DE000031B9A423ED814444FF00009D5E9003233
:103DF000C8F81C4013605A60C5F80090D8F810301D
:103E0000B34201D101F056FD89F31188D5E90331A0
:103E100028469847302383F311886B69002BD8D04C
:103E200001F038FD6A69A0EB040982464A450DD2CB
:103E3000022001F0B5FD0022D8F81030B34208D1BD
:103E400051462846BDE8F047FFF728BF121A224422
:103E5000F2E712EB09092946384638BF4A46FFF710
:103E6000EBFEB5E7D8F81030B34208D01444C8F8D8
:103E70001C00211AA960BDE8F047FFF7F3BEBDE8BA
:103E8000F08700BF98290020882900200020704773
:103E9000FEE70000704700004FF0FF307047000061
:103EA00002290CD0032904D00129074818BF00209B
:103EB0007047032A05D8054800EBC2007047044844
:103EC00070470020704700BFA06600083C22002019
:103ED0005466000870B59AB005460846144601A914
:103EE00000F0C2F801A8FDF72DFB431C0022C6B26A
:103EF0005B001046C5E9003423700323023404F844
:103F0000013C01ABD1B202348E4201D81AB070BD6F
:103F100013F8011B013204F8010C04F8021CF1E74C
:103F200008B5302383F311880348FFF74BF80023CB
:103F300083F3118808BD00BFF82B002090F8803073
:103F400003F01F02012A07D190F881200B2A03D128
:103F50000023C0E91D3315E003F06003202B08D1D6
:103F6000B0F884302BB990F88120212A03D81F2A79
:103F700004D8FFF709B8222AEBD0FAE7034A4267D0
:103F800007228267C3670120704700BF33220020E9
:103F900007B5052917D8DFE801F01916031919200C
:103FA000302383F31188104A01210190FFF7B2F802
:103FB000019802210D4AFFF7ADF80D48FEF7CEFF3C
:103FC000002383F3118803B05DF804FB302383F3EF
:103FD00011880748FEF798FFF2E7302383F3118832
:103FE0000348FEF7AFFFEBE7F4650008186600082A
:103FF000F82B002038B50C4D0C4C2A460C4904F126
:104000000800FFF767FF05F1CA0204F11000094933
:10401000FFF760FF05F5CA7204F118000649BDE814
:104020003840FFF757BF00BFD04400203C2200209B
:10403000D4650008DE650008E965000870B504462F
:1040400008460D46FDF77EFAC6B2204601340378D5
:104050000BB9184670BD32462946FDF753FA0028C1
:10406000F3D10120F6E700002DE9F84F05460C4694
:10407000FDF768FA2C49C6B22846FFF7DFFF08B102
:104080000336F6B229492846FFF7D8FF08B11036A3
:10409000F6B2632E0DD8DFF89080DFF89090244FB1
:1040A000DFF894A0DFF894B02E7846B92670BDE80A
:1040B000F88F29462046BDE8F84F02F0FDB8252EBE
:1040C0002ED1072241462846FDF71CFA70B9DBF8CD
:1040D000003007350A3444F80A3CDBF8043044F871
:1040E000063CBBF8083024F8023CDDE708224946CC
:1040F0002846FDF707FA98B9A21C0E4B1978023230
:104100000909C95D02F8041C13F8011B01F00F0135
:104110005345C95D02F8031CF0D118340835C3E7D4
:10412000013504F8016BBFE7C0660008E9650008C7
:10413000D366000800E8F11F0CE8F11FC86600080C
:10414000BFF34F8F044B1A695107FCD1D3F81021EC
:104150005207F8D1704700BF0020005208B50D4B40
:104160001B78ABB9FFF7ECFF0B4BDA68D10704D52E
:104170000A4A5A6002F188325A60D3F80C21D207F9
:1041800006D5064AC3F8042102F18832C3F8042197
:1041900008BD00BF2E4700200020005223016745C4
:1041A0004FF00063054A1968013104D1043393428A
:1041B000F9D1012070470020704700BF00000208BD
:1041C00008B5114B1B78F3B9104B1A69510703D589
:1041D000DA6842F04002DA60D3F81021520705D5C0
:1041E000D3F80C2142F04002C3F80C21FFF7A8FFDE
:1041F000064BDA6842F00102DA60D3F80C2142F093
:104200000102C3F80C2108BD2E47002000200052F7
:104210004FF40030704700000120704708B9FFF7E5
:10422000BFBF00207047000038B548BB154CFFF7F2
:1042300053FCFFF785FF0546FFF790FF4FF0FF3374
:104240006361C4F814312361FFF77AFF2423E3602C
:10425000E36843F08003E36023695B07FCD4FFF766
:104260006FFF4FF000604FF4003100F007FA28466E
:10427000FFF7A6FFFFF73AFCBDE83840FFF790BF15
:10428000002038BD002000522DE9F84F40EA02031B
:1042900005460C461746D80602D00020BDE8F88F28
:1042A00027F01F07DFF8D4B0FFF758FF2744BC42C0
:1042B00003D10120FFF784FFF0E7202229462046A2
:1042C00001F0A6FF10B920352034F0E72B4605F1A8
:1042D00020021E68711CE0D104339A42F9D1FFF725
:1042E000FBFB05F17843234AB3F5801F224B28BF1F
:1042F0009A4603F1040338BF9046A2F1080228BF92
:104300009846A3F108033ABF9146DA469946FFF76B
:1043100017FFC8F80060A5EB040CD9F8002004F1E1
:104320001C0142F00202C9F80020221FDAF80060E6
:1043300016F00506FAD152F8043F8A424CF80230D2
:10434000F4D1BFF34F8FFFF7FBFE4FF0FF32C8F8F9
:104350000020D9F8002022F00202C9F80020FFF75F
:10436000C5FB20222146284601F052FF0028AAD092
:1043700030469FE7142000521021005210200052B6
:1043800010B5084C237828B11BB9FFF7E7FE0123CD
:10439000237010BD002BFCD02070BDE81040FFF74B
:1043A0000FBF00BF2E4700202DE9F74F0E460546F0
:1043B000002864D011F0050763D139B908222946D5
:1043C0003046FFF7B9F90446002848D108224FF0DB
:1043D0000109DFF8C08006F00403DFF8BCA006EA9C
:1043E000090BBBF1000F27D0D8F81410C80723D44D
:1043F00009F1010908F10C08B9F1060FF1D18FB9E3
:10440000224E2946F0190092FFF796F9044630BB78
:104410001837009A782FF4D12946FFF78DF9044612
:10442000E8B9009A29461A48FFF786F9044608BBFE
:10443000204603B0BDE8F08FABB1D8F8141011F0EE
:10444000040FD5D01820294600FB09A0CDE9002390
:10445000FFF772F90446DDE900230028C8D02A4698
:104460000021204608E0B107ECD5D8F8141011F06F
:10447000020FE6E72A460021FDF76CF8D8E704466C
:10448000D6E71F35202225F01F05A0E76047002052
:1044900030470020E4660008484700200021FFF76D
:1044A00083BF00000121FFF77FBF0000F8B5144D66
:1044B00001241827134E40F2FF3200210120FDF79E
:1044C00049F807FB046001342A6955F80C1FFFF70F
:1044D0001FF9062CF5D137254FF4C0542046FFF7BD
:1044E000E1FF014628B122460748BDE8F840FFF742
:1044F0000FB9C4EBC404013D4FEAD404EED1F8BDBA
:10450000E466000848470020304700200421FFF7F8
:104510004BBF00004843FFF7C1BF000008B1FFF7E1
:104520007DB9704738B5054D00240334696855F8E6
:104530000C0B00F0B5F8122CF7D138BDE46600087A
:1045400070B5104E82B0FFF7C7FA054601F0A2F928
:10455000326803469042336037BF0B4A0A495168BC
:10456000146836BF0131D1E9004151600419284671
:1045700041F100010191FFF7B9FA2046019902B01B
:1045800070BD00BFD8470020E047002070B5124E34
:1045900082B0FFF7A1FA054601F07CF932680346C4
:1045A0009042336037BF0D4A0C495168146836BFDA
:1045B0000131D1E9004151600419284641F100015F
:1045C0000191FFF793FA4FF47A7200232046019984
:1045D000FBF78EFE02B070BDD8470020E0470020F8
:1045E0000244074BD2B210B5904200D110BD441C1A
:1045F00000B253F8200041F8040BE0B2F4E700BF2A
:10460000504000580E4B30B51C6F240405D41C6F6D
:104610001C671C6F44F400441C670A4C0244236866
:10462000D2B243F480732360074B904200D130BD77
:10463000441C51F8045B00B243F82050E0B2F4E7A8
:1046400000440258004802585040005807B5012263
:1046500001A90020FFF7C4FF019803B05DF804FB37
:1046600013B50446FFF7F2FFA04205D0012201A9CD
:1046700000200194FFF7C6FF02B010BD0144BFF354
:104680004F8F064B884204D3BFF34F8FBFF36F8F1A
:104690007047C3F85C022030F4E700BF00ED00E093
:1046A0000144BFF34F8F064B884204D3BFF34F8FB3
:1046B000BFF36F8F7047C3F870022030F4E700BF7C
:1046C00000ED00E07047000070B5054616460C4648
:1046D00001201021FFF71EFF286046733CB12046E1
:1046E00036B1FFF713FF2B68186000B19C6070BDF6
:1046F000FFF7D8FEF7E7000070B50E4615460446F2
:1047000000B30B6843608368934210D213B1006812
:10471000FFF704FF637B28462BB1FFF7F7FE20600D
:1047200020B9A06070BDFFF7BDFEF8E7A560206866
:1047300005F11F01306021F01F01FFF79FFF0120ED
:104740002073EFE70120EDE710B5044640B10068A3
:10475000884205D1606808B1FCF7CAFE00232373C4
:1047600010BD000070B50E461546044620B38368A0
:104770009A4210D913B10068FFF7D0FE637B284638
:104780002BB1FFF7C3FE206020B9A06070BDFFF71A
:1047900089FEF8E7A560316819B12A462068FCF760
:1047A000A7FE206805F11F01306021F01F01FFF70F
:1047B00077FF01202073E9E70120E7E720B10368D4
:1047C0008B4204BF002303737047000008B100232D
:1047D00003737047034B1A681AB9034AD2F8D024FE
:1047E0001A607047E84700200040025808B5FFF7FC
:1047F000F1FF024B1868C0F3806008BDE847002055
:1048000070B5BFF34F8FBFF36F8F1A4A0021C2F804
:104810005012BFF34F8FBFF36F8F536943F40033D0
:104820005361BFF34F8FBFF36F8FC2F88410BFF394
:104830004F8FD2F8803043F6E074C3F3C900C3F35E
:104840004E335B0103EA0406014646EA81750139ED
:10485000C2F86052F9D2203B13F1200FF2D1BFF31E
:104860004F8F536943F480335361BFF34F8FBFF3CE
:104870006F8F70BD00ED00E0FEE700000A4B0B48B3
:104880000B4A90420BD30B4BC11EDA1C121A22F0BA
:1048900003028B4238BF00220021FCF75BBE53F8B5
:1048A000041B40F8041BECE7B0690008904A0020A4
:1048B000904A0020904A00207047000003681A6860
:1048C00099685A6043681BB142EA01418068184701
:1048D000704700004FF0A44310B51C68E00702D5F4
:1048E0002848FFF7EBFFA10702D52748FFF7E6FFAF
:1048F000620702D52548FFF7E1FF230702D52448C8
:10490000FFF7DCFFE00602D52248FFF7D7FFA1063C
:1049100002D52148FFF7D2FF620602D51F48FFF7F4
:10492000CDFF230602D51E48FFF7C8FFE00502D5DC
:104930001C48FFF7C3FFA10502D51B48FFF7BEFFC8
:10494000620502D51948FFF7B9FF230502D51848BB
:10495000FFF7B4FFE00402D51648FFF7AFFFA1044C
:1049600002D51548FFF7AAFF620402D51348FFF7E6
:10497000A5FF230402D51248FFF7A0FFBDE81040B1
:1049800001F000B9F0470020FC4700200848002053
:1049900014480020204800202C48002038480020DF
:1049A00044480020504800205C480020684800200F
:1049B00074480020804800208C480020984800203F
:1049C000A448002030B5094B0021094C10200725D0
:1049D000196054F8042B0138C3E90121D16003F1B7
:1049E0000C0311615560F4D130BD00BFEC470020CD
:1049F0002C6700080F28F0B50AD9102806D10F231C
:104A00000020144C01272568984203D900201DE09E
:104A10000346F6E707FA00F6354218D10C23354372
:104A200043432560181D2344C3E902120A4B204466
:104A3000D3F8D42042F00102C3F8D420D3F8FC20EC
:104A400042F00102C3F8FC20D3F8FC30F0BD013085
:104A5000DAE700BFEC470020004402580368D96839
:104A6000DA68C90722F03F02DA6002D51A689207B5
:104A7000FCD507225A607047074BD3F8D81021EABB
:104A80000001C3F8D810D3F8002122EA0002C3F8CD
:104A90000021D3F8003170470044025870B5D0E9C6
:104AA000244300224FF0FF359E6804EB421351016E
:104AB000D3F80009002805DAD3F8000940F0804057
:104AC000C3F80009D3F8000B002805DAD3F8000B6F
:104AD00040F08040C3F8000B013263189642C3F8DF
:104AE0000859C3F8085BE0D24FF00113C4F81C3832
:104AF00070BD0000890141F02001016103699B063E
:104B0000FCD41220FFF702B810B50A4C2046FEF77D
:104B1000DFFA094BC4F89030084BC4F89430084CC5
:104B20002046FEF7D5FA074BC4F89030064BC4F880
:104B3000943010BDB0480020000008409067000885
:104B40004C490020000004409C67000870B50378C1
:104B50000546012B5CD1434BD0F89040984258D188
:104B6000414B0E216520D3F8D82042F00062C3F8F3
:104B7000D820D3F8002142F00062C3F80021D3F816
:104B80000021D3F8802042F00062C3F88020D3F8DF
:104B9000802022F00062C3F88020D3F8803000F03B
:104BA00097FC324BE360324BC4F800380023D5F851
:104BB0009060C4F8003EC02323604FF40413A36345
:104BC0003369002BFCDA01230C203361FEF79EFFD2
:104BD0003369DB07FCD41220FEF798FF3369002B02
:104BE000FCDA00262846A660FFF758FF6B68C4F879
:104BF0001068DB68C4F81468C4F81C6883BB1D4BDC
:104C0000A3614FF0FF336361A36843F00103A36026
:104C100070BD194B9842C9D1134B4FF08060D3F847
:104C2000D82042F00072C3F8D820D3F8002142F017
:104C30000072C3F80021D3F80021D3F8802042F09D
:104C40000072C3F88020D3F8802022F00072C3F8ED
:104C50008020D3F88030FFF70FFF0E214D209EE714
:104C6000064BCDE7B04800200044025840140040F5
:104C700003002002003C30C04C490020083C30C0FA
:104C8000F8B5D0F89040054600214FF00066204668
:104C9000FFF730FFD5F8941000234FF001128F6812
:104CA0004FF0FF30C4F83438C4F81C2804EB43122A
:104CB00001339F42C2F80069C2F8006BC2F80809CC
:104CC000C2F8080BF2D20B68D5F89020C5F89830DE
:104CD000636210231361166916F01006FBD11220CF
:104CE000FEF714FFD4F8003823F4FE63C4F800384C
:104CF000A36943F4402343F01003A3610923C4F8DC
:104D00001038C4F814380B4BEB604FF0C043C4F8B4
:104D1000103B094BC4F8003BC4F81069C4F80039D3
:104D2000D5F8983003F1100243F48013C5F89820A9
:104D3000A362F8BD6C67000840800010D0F8902096
:104D400090F88A10D2F8003823F4FE6343EA011386
:104D5000C2F80038704700002DE9F84300EB8103EA
:104D6000D0F890500C468046DA680FFA81F9480175
:104D7000166806F00306731E022B05EB41134FF075
:104D8000000194BFB604384EC3F8101B4FF0010168
:104D900004F1100398BF06F1805601FA03F39169FC
:104DA00098BF06F5004600293AD0578A04F1580109
:104DB000374349016F50D5F81C180B430021C5F843
:104DC0001C382B180127C3F81019A7405369611E1E
:104DD0009BB3138A928B9B08012A88BF5343D8F850
:104DE0009820981842EA034301F140022146C8F88E
:104DF0009800284605EB82025360FFF77BFE08EB24
:104E00008900C3681B8A43EA845348341E43640103
:104E10002E51D5F81C381F43C5F81C78BDE8F8831F
:104E200005EB4917D7F8001B21F40041C7F8001B18
:104E3000D5F81C1821EA0303C0E704F13F030B4A2D
:104E40002846214605EB83035A60FFF753FE05EB26
:104E50004910D0F8003923F40043C0F80039D5F8E0
:104E60001C3823EA0707D7E700800010000400027F
:104E7000D0F894201268C0F89820FFF70FBE000009
:104E80005831D0F8903049015B5813F4004004D0F9
:104E900013F4001F0CBF0220012070474831D0F8E6
:104EA000903049015B5813F4004004D013F4001F04
:104EB0000CBF02200120704700EB8101CB68196A0A
:104EC0000B6813604B6853607047000000EB810370
:104ED00030B5DD68AA691368D36019B9402B84BF67
:104EE000402313606B8A1468D0F890201C4402EBB6
:104EF0004110013C09B2B4FBF3F46343033323F0E4
:104F0000030343EAC44343F0C043C0F8103B2B689B
:104F100003F00303012B0ED1D2F8083802EB411045
:104F200013F4807FD0F8003B14BF43F0805343F06C
:104F30000053C0F8003B02EB4112D2F8003B43F0B3
:104F40000443C2F8003B30BD2DE9F041D0F8906039
:104F500005460C4606EB4113D3F8087B3A07C3F825
:104F6000087B08D5D6F814381B0704D500EB81035D
:104F7000DB685B689847FA071FD5D6F81438DB075B
:104F80001BD505EB8403D968CCB98B69488A5A686C
:104F9000B2FBF0F600FB16228AB91868DA68904274
:104FA0000DD2121AC3E90024302383F3118821465D
:104FB0002846FFF78BFF84F31188BDE8F0810123B9
:104FC00003FA04F26B8923EA02036B81CB68002B9E
:104FD000F3D021462846BDE8F041184700EB810395
:104FE0004A0170B5DD68D0F890306C692668E660DB
:104FF00056BB1A444FF40020C2F810092A6802F088
:105000000302012A0AB20ED1D3F8080803EB4214B6
:1050100010F4807FD4F8000914BF40F0805040F0B5
:105020000050C4F8000903EB4212D2F8000940F026
:105030000440C2F800090122D3F8340802FA01F151
:105040000143C3F8341870BD19B9402E84BF402005
:10505000206020681A442E8A8419013CB4FBF6F4BF
:1050600040EAC44040F00050C6E700002DE9F84394
:10507000D0F8906005460C464F0106EB4113D3F87B
:10508000088918F0010FC3F808891CD0D6F8103829
:10509000DB0718D500EB8103D3F80CC0DCF8143023
:1050A000D3F800E0DA68964530D2A2EB0E024FF05A
:1050B00000091A60C3F80490302383F31188FFF7C6
:1050C0008DFF89F3118818F0800F1DD0D6F8343881
:1050D0000126A640334217D005EB84030134D5F8EE
:1050E0009050D3F80CC0E4B22F44DCF8142005EB48
:1050F0000434D2F800E05168714514D3D5F834383F
:1051000023EA0606C5F83468BDE8F883012303FAEC
:1051100001F2038923EA02030381DCF80830002B43
:10512000D1D09847CFE7AEEB0103BCF81000834223
:1051300028BF0346D7F8180980B2B3EB800FE3D835
:105140009068A0F1040959F8048FC4F80080A0EB1E
:1051500009089844B8F1040FF5D818440B4490603E
:105160005360C8E72DE9F84FD0F8905004466E69B7
:10517000AB691E4016F480586E6103D0BDE8F84F4D
:10518000FEF716B8002E12DAD5F8003E9F0705D0BC
:10519000D5F8003E23F00303C5F8003ED5F80438E7
:1051A000204623F00103C5F80438FEF72DF830053A
:1051B00005D52046FFF772FC2046FEF715F8B1042E
:1051C0000CD5D5F8083813F0060FEB6823F47053AC
:1051D0000CBF43F4105343F4A053EB60320704D5E3
:1051E0006368DB680BB120469847F30200F1BA8090
:1051F000B70226D5D4F8909000274FF0010A09EBAA
:105200004712D2F8003B03F44023B3F5802F11D1AD
:10521000D2F8003B002B0DDA62890AFA07F322EA82
:105220000303638104EB8703DB68DB6813B1394652
:10523000204698470137D4F89430FFB29B689F42CC
:10524000DDD9F00619D5D4F89000026AC2F30A1726
:1052500002F00F0302F4F012B2F5802F00F0CA80C2
:10526000B2F5402F09D104EB8303002200F58050F2
:10527000DB681B6A974240F0B0803003D5F81858BD
:1052800035D5E90303D500212046FFF75DFEAA03CB
:1052900003D501212046FFF757FE6B0303D50221FA
:1052A0002046FFF751FE2F0303D503212046FFF7C9
:1052B0004BFEE80203D504212046FFF745FEA90274
:1052C00003D505212046FFF73FFE6A0203D50621DC
:1052D0002046FFF739FE2B0203D507212046FFF7B2
:1052E00033FEEF0103D508212046FFF72DFE7003A2
:1052F00040F1A780E90703D500212046FFF7B6FE5D
:10530000AA0703D501212046FFF7B0FE6B0703D59E
:1053100002212046FFF7AAFE2F0703D503212046CE
:10532000FFF7A4FEEE0603D504212046FFF79EFEFC
:10533000A80603D505212046FFF798FE690603D588
:1053400006212046FFF792FE2A0603D507212046B4
:10535000FFF78CFEEB0574D520460821BDE8F84F19
:10536000FFF784BED4F890904FF0000B4FF0010A85
:10537000D4F894305FFA8BF79B689F423FF638AFC2
:1053800009EB4713D3F8002902F44022B2F5802F2D
:1053900020D1D3F80029002A1CDAD3F8002942F0E2
:1053A0009042C3F80029D3F80029002AFBDB3946D4
:1053B000D4F89000FFF79EFB22890AFA07F322EA4D
:1053C0000303238104EB8703DB689B6813B1394631
:1053D000204698470BF1010BCAE7910701D1D0F89D
:1053E0000080072A02F101029CBF03F8018B4FEAFB
:1053F00018283FE704EB830300F58050DA68D2F801
:1054000018C0DCF80820DCE9001CA1EB0C0C002122
:105410008F4208D1DB689B699A683A449A605A685F
:105420003A445A6029E711F0030F01D1D0F8008007
:105430008C4501F1010184BF02F8018B4FEA182865
:10544000E6E7BDE8F88F000008B50348FFF78AFEDD
:10545000BDE8084000F096BBB048002008B50348FE
:10546000FFF780FEBDE8084000F08CBB4C490020EF
:10547000D0F8903003EB4111D1F8003B43F4001316
:10548000C1F8003B70470000D0F8903003EB4111A9
:10549000D1F8003943F40013C1F800397047000017
:1054A000D0F8903003EB4111D1F8003B23F4001306
:1054B000C1F8003B70470000D0F8903003EB411179
:1054C000D1F8003923F40013C1F800397047000007
:1054D000090100F16043012203F56143C9B283F879
:1054E000001300F01F039A4043099B0003F160433F
:1054F00003F56143C3F880211A60704730B5043367
:10550000039C0172002104FB0325C160C0E906531E
:10551000049B0363059BC0E90000C0E90422C0E9C5
:105520000842C0E90A11436330BD00000022416A0D
:10553000C260C0E90411C0E90A226FF00101FEF760
:105540006DBB0000D0E90432934201D1C2680AB9B0
:10555000181D704700207047036919600021C26858
:105560000132C260C269134482699342036124BF5D
:10557000436A0361FEF746BB38B504460D46E3684F
:105580003BB162690020131D1268A3621344E362F9
:1055900007E0237A33B929462046FEF723FB00288B
:1055A000EDDA38BD6FF00100FBE70000C368C269A7
:1055B000013BC3604369134482699342436124BF42
:1055C000436A436100238362036B03B1184770474A
:1055D00070B53023044683F31188866A3EB9FFF71D
:1055E000CBFF054618B186F31188284670BDA36A23
:1055F000E26A13F8015B9342A36202D32046FFF7ED
:10560000D5FF002383F31188EFE700002DE9F84F61
:1056100004460E46174698464FF0300989F3118824
:105620000025AA46D4F828B0BBF1000F09D14146A5
:105630002046FFF7A1FF20B18BF311882846BDE873
:10564000F88FD4E90A12A7EB050B521A934528BF2D
:105650009346BBF1400F1BD9334601F1400251F88C
:10566000040B914243F8040BF9D1A36A403640354C
:105670004033A362D4E90A239A4202D32046FFF7BB
:1056800095FF8AF31188BD42D8D289F31188C9E702
:1056900030465A46FBF72CFFA36A5E445D445B44E8
:1056A000A362E7E710B5029C0433017203FB0421F7
:1056B000C460C0E906130023C0E90A33039B0363F7
:1056C000049BC0E90000C0E90422C0E9084243632A
:1056D00010BD0000026A6FF00101C260426AC0E9B9
:1056E00004220022C0E90A22FEF798BAD0E9042376
:1056F0009A4201D1C26822B9184650F8043B0B60A7
:105700007047002070470000C3680021C269013360
:10571000C3604369134482699342436124BF436A6F
:105720004361FEF76FBA000038B504460D46E368E2
:105730003BB1236900201A1DA262E2691344E362AF
:1057400007E0237A33B929462046FEF74BFA0028B2
:10575000EDDA38BD6FF00100FBE700000369196066
:10576000C268013AC260C26913448269934203610C
:1057700024BF436A036100238362036B03B11847AC
:105780007047000070B530230D460446114683F380
:105790001188866A2EB9FFF7C7FF10B186F311880A
:1057A00070BDA36A1D70A36AE26A01339342A362CB
:1057B00004D3E16920460439FFF7D0FF002080F3CD
:1057C0001188EDE72DE9F84F04460D4690469946BD
:1057D0004FF0300A8AF311880026B346A76A4FB902
:1057E00049462046FFF7A0FF20B187F311883046D5
:1057F000BDE8F88FD4E90A073A1AA8EB06079742E2
:1058000028BF1746402F1BD905F1400355F8042B3C
:105810009D4240F8042BF9D1A36A40364033A3627D
:10582000D4E90A239A4204D3E16920460439FFF7F8
:1058300095FF8BF311884645D9D28AF31188CDE7BD
:1058400029463A46FBF754FEA36A3D443E443B4496
:10585000A362E5E7D0E904239A4217D1C3689BB15C
:10586000836A8BB1043B9B1A0ED01360C368013B63
:10587000C360C3691A4483699A42026124BF436AC0
:105880000361002383620123184670470023FBE76E
:1058900000F0A2B9014B586A704700BF000C0040ED
:1058A000034B002258631A610222DA60704700BF7E
:1058B000000C0040014B0022DA607047000C0040F1
:1058C000014B5863704700BF000C0040024B034A75
:1058D0001A60034A5A607047004A0020904A00202C
:1058E00000000220074B494210B55C68201A0840AE
:1058F0001968821A8A4203D3A24201D85A6010BDA5
:105900000020FCE7004A002008B5302383F311880B
:10591000FFF7E8FF002383F3118808BDFEE70000CE
:1059200070B51B4B0025044686B058600E46856254
:10593000016300F0FFF804F11003A560E562C4E91B
:1059400004334FF0FF33C4E90044C4E90635FFF7E0
:10595000A1FF2B46024604F134012046C4E9082386
:1059600080230C4A2565FEF7DBF801230A4AE06034
:1059700000920375684672680192B268CDE902230D
:10598000064BCDE90435FEF7F3F806B070BD00BF55
:10599000F02B0020A8670008AD6700081D5900081B
:1059A000024AD36A1843D062704700BF882900209A
:1059B0004B6843608B688360CB68C3600B6943614D
:1059C0004B6903628B6943620B6803607047000098
:1059D00008B5354B40F2FF70D3F8E0100143C3F82F
:1059E000E010D3F8082102433048C3F80821304AB8
:1059F000D3F808311146FFF7DBFF00F5806002F1B4
:105A00001C01FFF7D5FF00F5806002F13801FFF7B8
:105A1000CFFF00F5806002F15401FFF7C9FF00F5E8
:105A2000806002F17001FFF7C3FF00F5806002F1B2
:105A30008C01FFF7BDFF00F5806002F1A801FFF7C0
:105A4000B7FF00F5806002F1C401FFF7B1FF00F578
:105A5000806002F1E001FFF7ABFF00F5806002F12A
:105A6000FC01FFF7A5FF02F58C7100F58060FFF7E0
:105A70009FFF00F079F90F4BD3F8902242F001021A
:105A8000C3F89022D3F8942242F00102C3F8942282
:105A90000522C3F898204FF06052C3F89C20064AB4
:105AA000C3F8A02008BD00BF0044025800000258FF
:105AB000B467000800ED00E01F00080308B500F01F
:105AC0004BFBFDF7DDFF104BD3F8DC2042F040022A
:105AD000C3F8DC20D3F8042122F04002C3F80421EB
:105AE000D3F80431094B1A6842F008021A601A68A8
:105AF00042F004021A60FEF76DFEFEF7D7FCBDE827
:105B00000840FEF777BA00BF004402580018024868
:105B100070470000EFF30983054968334A6B22F0B0
:105B200001024A6383F30988002383F311887047D5
:105B300000EF00E0302080F3118862B60D4B0E4A72
:105B4000D96821F4E0610904090C0A430B49DA60C1
:105B5000D3F8FC2042F08072C3F8FC20084AC2F857
:105B6000B01F116841F0010111602022DA7783F83B
:105B70002200704700ED00E00003FA0555CEACC5E9
:105B8000001000E0302310B583F311880E4B5B68E2
:105B900013F4006314D0F1EE103AEFF309844FF0E0
:105BA0008073683CE361094BDB6B236684F30988EF
:105BB000FDF7FEFE10B1064BA36110BD054BFBE7E0
:105BC00083F31188F9E700BF00ED00E000EF00E08B
:105BD000470700084A070008114BD3F8E82042F0B5
:105BE0000802C3F8E820D3F8102142F00802C3F8F5
:105BF00010210C4AD3F81031D36B43F00803D36360
:105C0000EF22094B9A624FF0FF32DA6200229A616A
:105C10005A63DA605A6001225A611A60704700BF05
:105C2000004402580010005C000C0040094A08B50E
:105C30001169D3680B40D9B29B076FEA010111616A
:105C400007D5302383F31188FDF744FF002383F346
:105C5000118808BD000C0040064BD3F8DC2002433D
:105C6000C3F8DC20D3F804211043C3F80401D3F8AF
:105C7000043170470044025808B54FF0FF31394BEA
:105C8000D3F88020C3F88010D3F880200022C3F816
:105C90008020D3F88000D3F88400C3F88410D3F8B0
:105CA0008400C3F88420D3F88400D86F40F0FF400C
:105CB00040F4FF0040F4DF4040F07F00D867D86F29
:105CC00020F0FF4020F4FF0020F4DF4020F07F00B0
:105CD000D867D86FD3F888006FEA40506FEA505009
:105CE000C3F88800D3F88800C0F30A00C3F888001E
:105CF000D3F88800D3F89000C3F89010D3F8900040
:105D0000C3F89020D3F89000D3F89400C3F894100F
:105D1000D3F89400C3F89420D3F89400D3F89800F3
:105D2000C3F89810D3F89800C3F89820D3F89800D7
:105D3000D3F88C00C3F88C10D3F88C00C3F88C20F7
:105D4000D3F88C00D3F89C00C3F89C10D3F89C10B7
:105D5000C3F89C20D3F89C30FEF734FEBDE8084021
:105D600000F0CAB90044025808B50122564BC3F8E6
:105D70000821564BD3F8F42042F00202C3F8F42075
:105D8000D3F81C2142F00202C3F81C210222D3F8EE
:105D90001C314F4BDA605A689104FCD54D4A4E498C
:105DA0001A6001229A60D960002119614FF44041C4
:105DB00099614A4BDA6203F511339A699204FCD572
:105DC0001A6842F480721A60404B1A6F12F4407FD6
:105DD00004D04FF480321A6700221A671A6842F022
:105DE00001021A60394B1A685007FCD500221A616B
:105DF0001A6912F03802FBD1012119604FF080417D
:105E000059604FF00051D9605A67354ADA62354A15
:105E10001A611A6842F480321A602C4B1A68910396
:105E2000FCD51A6842F480521A601A689204FCD5B4
:105E30002D4A2E499A6200225A63196301F57A01AC
:105E4000DA6301F2D31199635A64294A1A64294A20
:105E5000DA621A6842F0A8521A601C4B1A6802F003
:105E60002852B2F1285FF9D148229A614FF4886232
:105E7000DA6140221A62204ADA64204A1A65204A0E
:105E80005A65204A9A6534231F4A1360136803F049
:105E90000F03042BFAD10D4A136943F00303136176
:105EA000136903F03803182BFAD14FF00050FFF7B5
:105EB000D3FE4FF08040FFF7CFFE4FF00040BDE82B
:105EC0000840FFF7C9BE00BF0080005100440258DF
:105ED0000048025800C000F0020000010004005811
:105EE0000000FF01008890081210200077020B01CB
:105EF000470E0508DD0BBF01200000200000011047
:105F00000910E00000010110002000524FF0B042E3
:105F100008B5D2F8883003F00103C2F8883023B105
:105F2000044A13680BB150689847BDE80840FFF772
:105F300029BE00BF084A00204FF0B04208B5D2F891
:105F4000883003F00203C2F8883023B1044A936812
:105F50000BB1D0689847BDE80840FFF713BE00BFFB
:105F6000084A00204FF0B04208B5D2F8883003F05C
:105F70000403C2F8883023B1044A13690BB1506995
:105F80009847BDE80840FFF7FDBD00BF084A002064
:105F90004FF0B04208B5D2F8883003F00803C2F8D9
:105FA000883023B1044A93690BB1D0699847BDE8A2
:105FB0000840FFF7E7BD00BF084A00204FF0B0429D
:105FC00008B5D2F8883003F01003C2F8883023B146
:105FD000044A136A0BB1506A9847BDE80840FFF7BE
:105FE000D1BD00BF084A00204FF0B04310B5D3F830
:105FF000884004F47872C3F88820A30604D5124AB6
:10600000936A0BB1D06A9847600604D50E4A136BA9
:106010000BB1506B9847210604D50B4A936B0BB11B
:10602000D06B9847E20504D5074A136C0BB1506C4E
:106030009847A30504D5044A936C0BB1D06C9847DC
:10604000BDE81040FFF79EBD084A00204FF0B04366
:1060500010B5D3F8884004F47C42C3F88820620568
:1060600004D5164A136D0BB1506D9847230504D51E
:10607000124A936D0BB1D06D9847E00404D50F4AD6
:10608000136E0BB1506E9847A10404D50B4A936E62
:106090000BB1D06E9847620404D5084A136F0BB158
:1060A000506F9847230404D5044A936F0BB1D06F07
:1060B0009847BDE81040FFF765BD00BF084A0020C3
:1060C00008B50348FCF75EFBBDE80840FFF75ABD82
:1060D000E024002008B50348FCF706FCBDE80840B2
:1060E000FFF750BD0025002008B5FFF79FFDBDE874
:1060F0000840FFF747BD0000062108B50846FFF736
:10610000E7F906210720FFF7E3F906210820FFF74A
:10611000DFF906210920FFF7DBF906210A20FFF746
:10612000D7F906211720FFF7D3F906212820FFF71A
:10613000CFF909217A20FFF7CBF90A215C20FFF77C
:10614000C7F907213220FFF7C3F90C212520BDE84C
:106150000840FFF7BDB9000008B5FFF78DFD00F05E
:106160000FF8FCF7D9FDFCF7B1FFFCF783FEFDF754
:1061700043FAFFF7CDFCBDE80840FFF789BB0000FC
:106180000023054A19460133102BC2E9001102F120
:106190000802F8D1704700BF084A00200B460146AC
:1061A000184600F027B80000FEF7B8B9FFF7FCBFAB
:1061B000012838BF012010B504462046FEF76EF9CD
:1061C00030B900F007F808B900F00CF88047F4E7A0
:1061D00010BD0000024B1868BFF35B8F704700BF13
:1061E000884A002008B5062000F04AF80120FDF793
:1061F0004FFE000010B5054C13462CB10A4601466F
:106200000220AFF3008010BD2046FCE70000000034
:1062100010B501390244904201D1002005E0037815
:1062200011F8014FA34201D0181B10BD0130F2E755
:106230001F2938B504460D4604D9162303604FF0D4
:10624000FF3038BD426C12B152F821304BB92046B4
:1062500000F030F82A4601462046BDE8384000F0FC
:1062600017B8012B0AD0591C03D116230360012053
:10627000E7E7002442F82540284698470020E0E759
:10628000024B01461868FFF7D3BF00BF5C22002015
:1062900038B5074D00230446084611462B60FDF72C
:1062A000FBFD431C02D12B6803B1236038BD00BF46
:1062B0008C4A0020FDF7EABD034611F8012B03F8D4
:1062C000012B002AF9D170470000000001000000F6
:1062D00000010001000000000000000000000000BC
:1062E00052657175657374656420746F20657261A1
:1062F0007365206D6F7265207468616E207765200C
:1063000063616E0A00457261736520436F6D6D6154
:106310006E642052656365697665640A0050435473
:1063200020444F4E453A2025640A000053544D3313
:106330003248373F3F3F0053544D333248373433B0
:106340002F37353300000000F82B002000250020F7
:10635000773235712D647472000000000000000077
:106360000000000000000000000000004D170008C1
:10637000B11A0008B11A0008511700085517000893
:10638000591700085D170008B11A0008B11A000873
:10639000B11A00087517000879170008911700084E
:1063A00099170008A5170008A9170008AD170008DD
:1063B000E0240020010000000000000000000000B8
:1063C000CD180008E51800084D170008B917000897
:1063D00019190008D5170008B1190008E1190008BB
:1063E0005D170008D1170008BD170008CD17000879
:1063F0007517000879170008911700089917000809
:10640000A5170008A9170008AD1700080000000034
:10641000000000004D180008B1170008B51700086B
:1064200053464450000000004A454445433A204644
:1064300061696C656420746F2064657465637420A1
:10644000666C617368206465766963653A202573BC
:106450000A004A454445433A204661696C65642018
:10646000746F20636F6E66696720666C6173682065
:106470006465766963653A2025730A004A45444598
:10648000433A20446574656374656420466C6173A7
:1064900068204465766963653A2025730A0045786B
:1064A0007420466C617368204E6F7420466F756E61
:1064B000642100006D74323571007732357100004F
:1064C000B464000820BA0000BA640008EF4000007D
:1064D00050630008EF7000000000000000000000A2
:1064E00091210008F1230008CD1A0008D11A0008F4
:1064F000791B000859230008D51A0008D91A00088A
:1065000051220008491B0008B1220008B51F0008ED
:10651000E11A0008DD1A000881240008411B000868
:106520000000000000000000452500084D2500087F
:1065300031250008392500085D250008612500087F
:106540004D444D41206661696C7572650000000024
:1065500000960000000000000000000000000000A5
:10656000000000000000000000000000D92C00081E
:10657000C52C0008012D0008ED2C0008F92C00089E
:10658000E52C0008D12C0008BD2C00080D2D0008BA
:1065900000000000F12D0008DD2D0008192E000874
:1065A000052E0008112E0008FD2D0008E92D000819
:1065B000D52D0008252E0008000000000100000075
:1065C0000000000063300000C4650008E0290020DE
:1065D000F02B00204172647550696C6F7400254285
:1065E0004F415244252D424C002553455249414CC0
:1065F000250000000200000000000000113000082B
:106600008130000840004000A0440020B044002039
:106610000200000000000000030000000000000075
:10662000C93000080000000010000000C044002035
:10663000000000000100000000000000B048002041
:1066400001010200913F0008A13E00083D3F000803
:10665000213F0008430000005C6600080902430077
:10666000020100C0320904000001020201000524F9
:106670000010010524010001042402020524060083
:1066800001070582030800FF09040100020A000057
:1066900000070501024000000705810240000000DC
:1066A00012000000A866000812011001020000405C
:1066B000091241570002010203010000040309040A
:1066C00025424F41524425005350526163696E6721
:1066D0004837003031323334353637383941424368
:1066E00044454600000000200000020002000000B7
:1066F0000000003000000400000000000000002442
:1067000000000800040000000004000000FC00007D
:1067100002000000000004300080000000000000C3
:10672000000000380000010001000000400000529D
:1067300080000052C000005200010052400100528F
:1067400080010052C001005200020052400200527B
:1067500080020052C0020052000300524003005267
:1067600080030052C00300520004005200000000E9
:106770001D320008D5340008813500084000400073
:10678000E8490020E849002001000000F849002005
:10679000800000004001000008000000000100002F
:1067A00000040000080000006D61696E0069646CFF
:1067B000650000000000806A00000000AAAAAAAAE2
:1067C00000000064FFFF00000000000000A00A00BD
:1067D000240020A100000000BAAABAAA00000051BB
:1067E000FFFF000000090000000900440000000055
:1067F00000000000AAAAAAAA00000000FFFF0000F3
:1068000000000000000000000000800A00000000FE
:10681000AAAAEAAF00000000FFFF0000000000008D
:10682000009099006000400000000000BAAAAAAAE7
:1068300000004000F7FF0000000900000000000019
:106840000000000000000000AAAAAAAA00000000A0
:10685000FFFF00000000000000000000000000003A
:1068600000000000AAAAAAAA00000000FFFF000082
:106870000000000000000000000000000000000018
:10688000AAAAAAAA00000000FFFF00000000000062
:10689000000000000000000000000000AAAAAAAA50
:1068A00000000000FFFF00000000000000000000EA
:1068B0000000000000000000AAAAAAAA0000000030
:1068C000FFFF0000000000000000000000000000CA
:1068D00000000000AAAAAAAA00000000FFFF000012
:1068E0000000000000000000389AFF7F0100000057
:1068F0002404000000000000000000000000E90087
:10690000FF000000000000002C6300083F000000B2
:1069100050040000376300083F00000000960000AC
:1069200000000800960000000008000004000000BD
:10693000BC6600080000000000000000000000002D
:1069400000000000000000000000000060220020A5
:106950000000000000000000000000000000000037
:106960000000000000000000000000000000000027
:106970000000000000000000000000000000000017
:106980000000000000000000000000000000000007
:1069900000000000000000000000000000000000F7
:1069A00000000000000000000000000000000000E7
:00000001FF
